:100000000C9442040C946A040C946A040C946A04E0
:100010000C946A040C946A040C946A040C946A04A8
:100020000C946A040C9443050C940C290C94293804
:100030000C946A040C94E6350C9424360C946A04EF
:100040000C946A040C946A040C946A040C946A0478
:100050000C946A04000000000067582F00000000A4
:10006000F567E630C80232002F2CE8031009320091
:10007000802F2C01000000000000000000000000A4
:1000800000000000000000002ECA7E3BC24CA40B02
:100090000C4970170000000043BFA80E00000000CC
:1000A00080D566100000000080D0841F0000000092
:1000B00031D5611000000000C0D6651000000000BE
:1000C00080D465100000000080D46510C6023200A4
:1000D0002E2CE80304013200D2052C010006080092
:1000E00001FF010100000106090001FF03020100F8
:1000F00002060A0001FF0000000006060E0000FFD5
:100100000302010005060D0000FF020300000406C3
:100110000C0000FF0302010003060B0000FF0406B1
:1001200000000706070000FF030201009F0D9A0D63
:10013000E50E2020436865616C69436861726765FC
:100140007200202020207665723A20302E33320053
:10015000540100006F7074696F6E7300010001003C
:100160000100010001000A00640001000200040017
:100170001000400000010004010003000800070017
:10018000070014000700496E660079657300206E51
:100190006F006D560047024F02540259025D026221
:1001A0000267026C0201000100010001000000B0C2
:1001B000041C07520300000807B0044006E80300CF
:1001C000000807D0079209D60600000000E40C10D2
:1001D0000ED007E40C0000100E0410C409A60E0097
:1001E00000740E6810B80B0A0F000040066C07146C
:1001F000054006000000980898086C071027019831
:100200000898086C07010002980898086C0701001C
:10021000039808DC006C07060004980898086C072F
:10022000030005980898086C0703000698089808CA
:100230006C07030007980898086C070300756E6C3C
:10024000696D6974656400556E6B6E6F776E004EF4
:10025000694364004E694D480050623F004C696636
:1002600065004C696C6F004C69706F004E695A6E86
:1002700000920299029E02A302A802AD02BB0200F4
:100280000045646974206E616D653A004E616D656C
:100290003A004261743A202000563A202000436818
:1002A0003A200049633A200049643A200020206344
:1002B0007265617465206E616D6500202020656443
:1002C0006974206E616D650043684342426C446905
:1002D00046435374534243684469437943594368DE
:1002E000446945420020202D2D2020006E2E612ED5
:1002F000004C696D6974733A200074696D653A2029
:100300002020202000622000202000626174742ED2
:1003100020523D00776972657320523D0056696E28
:100320007075743D00206C696D69743D00566F7581
:1003300074203D005662616C2E3D00546578743D1A
:10034000002D0070726F6772616D20636F6D706C4D
:1003500065746500726561736F6E3A20006D6F6E33
:1003600069746F72206572726F72006E6F7420759F
:10037000736564006D6178566F75743D0064656CDB
:10038000746120563D2000546578743D006E6F7492
:1003900020757365640064656C746120543D2000B1
:1003A00046756E6374696F6E206E6F7400696D7050
:1003B0006C656D656E7465642079657400706C653C
:1003C0006173652063616C69627261746500626566
:1003D000666F7265207573650052455645525345E8
:1003E00020504F4C41524954590046554C2000254D
:1003F0002000AD20A120B12056206C696D697400E9
:100400002D64560064542F64740076217F214221AC
:10041000A721AE21ED2152222022262201230F23E3
:100420008322010607050002060708090B0C0D04CC
:1004300005030002060708090B0C0D040503000262
:100440000A0E0F0B0C0D0405030002060708090B2A
:100450000C0D04050300020F0B0C0D040503000630
:10046000070405000000010203040D00010203045B
:1004700005060D0708090A0D0B0C0DAF04B604C5DF
:1004800004CD04D704E304EB04FA040000AF04CD68
:100490000407051105FA040000AF04B604C504CD35
:1004A00004D704FA040000AF04CD04FA040000638A
:1004B0006861726765006368617267652B62616C71
:1004C000616E63650062616C616E6365006469738F
:1004D0006368617267650066617374206368617246
:1004E00067650073746F726167650073746F726122
:1004F00067652B62616C616E63006564697420627C
:1005000061747465727900633E64206379636C651D
:1005100000643E63206379636C65006261742064EB
:1005200069736300696E7075742056006361702092
:10053000434F4646006578742054434F4600436F4E
:100540006E6E65637420426174746572792100B7C0
:1005500005C005C905000008090A08090AD205D81E
:1005600005DE05E405EA05F005F605FC05020600D2
:1005700000061E1F20212223120006090A0B0C0D63
:100580000E76616C75653A2000496F75743A2020CB
:100590000008060D0600000806140600001A0621D1
:1005A0000600002806310600003A0642064B0657B0
:1005B0000663066F06000056623070696E3A2000CE
:1005C00056623170696E3A200056623270696E3A36
:1005D000200056696E3A20005662313A2000566279
:1005E000323A20005662333A20005662343A2000F4
:1005F0005662353A20005662363A200056312D3682
:100600003A00566F75743A0035306D410031303024
:10061000306D41003330306D410074656D703A20AB
:100620000076616C75653A00706F696E7420312ECA
:1006300000706F696E7420322E00766F6C74616783
:1006400065004920636861726765004920646973C9
:100650006368617267650074656D702065787465A4
:10066000726E0063616C69622D3E554152540065A3
:1006700078706572742044414E47455221008606C9
:100680008F069906000073657474696E6773006362
:10069000616C69627261746500726573657420646F
:1006A000656661756C740080250000004B000000D9
:1006B00096000000E1000000C20100000070176415
:1006C0000007000C0005007800581B00000800001F
:1006D000000300FD06090714071B0725072F073B2A
:1006E0000745075007590763076A07720700004369
:1006F0002F6D007B0784078B0791079A0765787435
:10070000726E20543A20202000657874726E205456
:10071000434F3A0064542F64743A004E694D4820A8
:100720002D64563A004E694364202D64563A0043C6
:100730002F44206379636C65733A006361702043D2
:100740004F66663A00696E707574206C6F773A0078
:100750006469736368202B3A0062616C2E206572B5
:10076000723A00554152543A200073706565643AFC
:1007700020002020207265736574006469736162D3
:100780006C6564006E6F726D616C006465627567A4
:10079000006578742E20646562006578742E2041AF
:1007A00064630013161817190705061E1F2021225F
:1007B000237265736574696E6720656570726F6D0D
:1007C0003A00763A20372E312E3220006320006422
:1007D0002000732000000000000000000000000066
:1007E00000000403000500000000000000000000FD
:1007F00000000000000000000000000000000001F8
:1008000000000020408000000000000102040810E9
:1008100020408000000102040810204080000000F9
:1008200080402010080402010000010204081000AA
:100830000202020000000000040404040404040492
:10084000000003030303030303030000000101018D
:100850000101010101000002020202020000390050
:1008600036003300300000003B0038003500320015
:1008700000003A0037003400310030055210752076
:100880007325163711241FBECFE5D8E0DEBFCDBFDC
:1008900010E0A0E6B0E0EEE9F4E702C005900D92AA
:1008A000A83EB107D9F714E0A8EEB0E001C01D9250
:1008B000A33AB107E1F718E0C4E8D8E004C02297F2
:1008C000FE010E94D439CA37D107C9F70E94D23736
:1008D0000C944D3A0C940000CF9388E20E941D398D
:1008E000C1E0892B09F0C0E089E20E941D39892B03
:1008F00011F080E001C082E0C82B8AE20E941D391D
:10090000892B11F080E001C084E0C82B8BE20E94AB
:100910001D39892B11F080E001C088E08C2BCF912C
:100920000895CF93C82F682F89E10E94AE386C2FAD
:100930008AE10E94AE386C2F80E20E94AE386C2FA4
:1009400089E00E94AE386C2F8BE00E94AE386C2F8D
:1009500080E1CF910C94AE3808958091FD008823FA
:1009600031F08091FE008F5F8093FE0002C01092F4
:10097000FE008091FD008A3010F480E001C088E024
:100980009091FD00943108F084E09091FD009E313B
:1009900008F082E06091FE0068238CE20C94E63857
:1009A0008093FD00089561E068278CE00C94E638A0
:1009B00080E00E94263861E08CE00E94AE3861E061
:1009C0008EE00E94AE3861E08EE10E94AE3861E0B8
:1009D0008CE20E94AE3861E08DE00E94AE3861E0AA
:1009E0008EE00E94AE3861E08FE00E94AE3880E079
:1009F0000E94D3041092FD0020E042E060E188EE06
:100A000090E00E949D160E94D4280E9466230E94B6
:100A1000C7230E94B3050E947F070C94EC0CCF9370
:100A2000C82F682F617089E10E94E6386C2F6270D0
:100A30008AE10E94E6386C2F647080E20E94E638FA
:100A40006C2F687089E00E94E6386C2F60718BE033
:100A50000E94E6386C2F607280E1CF910C94E638EA
:100A6000CF92EF920F9383E1C82E94E1E92E05E136
:100A700026E147E168E188EE90E00E9451170F916E
:100A8000EF90CF9008951F920F920FB60F921124FE
:100A90002F933F934F935F936F937F938F939F9386
:100AA000AF93BF93EF93FF93209102013091030125
:100AB0008091000190910101820F931F9093010199
:100AC00080930001809100019091010126E09695AC
:100AD00087952A95E1F72091000130910101AC0141
:100AE00066E0440F551F6A95E1F7241B350B3093E0
:100AF0000101209300012FB7F8943091FF003E30A0
:100B000011F49BBD8ABD3091FF003D3021F02FBF15
:100B10000E94AD0403C099BD88BDF9CFFF91EF914C
:100B2000BF91AF919F918F917F916F915F914F9105
:100B30003F912F910F900FBE0F901F9018959FB768
:100B4000F89470930301609302018093FF008E304C
:100B500019F48FB5806804C08D3019F48FB58062A8
:100B60008FBD9FBF08951FBC80E18EBD2FB7F89445
:100B700080E091E097BD86BD2FBF8EB5887F8EBD8A
:100B80008EB581608EBD89B7846089BF08958E302F
:100B900019F48FB58F7704C08D3019F48FB58F7D20
:100BA0008FBD0895409105015091060160910701A4
:100BB00070910801452F562F672F772767FD7A958B
:100BC000CA01089510920C0110920B018617970725
:100BD00068F480E090E4A0E0B0E080930501909399
:100BE0000601A0930701B093080108C01092050107
:100BF00010920601109207011092080180910501E0
:100C000090910601A0910701B0910801BA2FA92F78
:100C1000982F88278093050190930601A0930701E0
:100C2000B093080181E0809304010895CF93DF938E
:100C3000EC01C13080E6D80770F4C13080E4D807F9
:100C400060F48EE00E94C70560E08EE00E94E63806
:100C5000BE018DE00CC0C0E0D0E68DE00E94C7056B
:100C600061E08DE00E94E638BE0170548EE0DF91B5
:100C7000CF910C949F0590930C0180930B016CEB2A
:100C800076E680E00E948E0C90930A018093090121
:100C90000895CF93C82F882319F080E00E9456064C
:100CA00061E06C278EE1CF910C94E638CF93DF930F
:100CB000C82F882319F080E00E9449068DE00E9429
:100CC000C70560E08DE00E94E6388EE00E94C7050F
:100CD00060E08EE00E94E6381092040161E06C272B
:100CE0008FE00E94E638CC2361F080E00E944B0840
:100CF000EC0186E00E944B08BE01DF91CF910C947D
:100D0000E205DF91CF9108950F931F938091040125
:100D1000882309F474C080E00E94540820910901DE
:100D200030910A012817390730F480E00E945606F6
:100D30001092040164C082E00E94540840910B01AB
:100D400050910C0160E070E00091050110910601E6
:100D50002091070130910801481B590B6109710965
:100D6000E4E0440F551F661F771FEA95D1F7040F83
:100D7000151F261F371F00930501109306012093AE
:100D80000701309308018091050190910601A0911F
:100D90000701B0910801B7FF08C010920501109239
:100DA00006011092070110920801809105019091AF
:100DB0000601A0910701B09108010197A046B10575
:100DC00060F080E090E0A0E6B0E0809305019093B1
:100DD0000601A0930701B09308018091050190914D
:100DE0000601A0910701B0910801892F9A2FAB2F1E
:100DF000BB27A7FDBA951F910F910C9416061F9162
:100E00000F910895BC018EE00C949F05877080625D
:100E100087B90895CF93DF9390916000891721F1EE
:100E200080936000C8B390E2899F90011124CF7134
:100E3000C22B98B3E1E2F8E0E4912AB3DE2FD0951B
:100E4000D2232AB38150823050F0892F8F71806C69
:100E500088BBE22BEABB8AE090E00E9473388FB730
:100E6000F894C8BBDABB8FBFDF91CF91089595E0AE
:100E7000899FF0011124E052FF4FE49181E0E111DC
:100E800001C080E0089595E0899FF0011124E152AE
:100E9000FF4FE49181E0E11101C080E0089524B1A9
:100EA00035B195E0899FF0011124E252FF4FE491A2
:100EB000F0E0EE0FFF1FEA54FE4F932F80E0822BED
:100EC00091838083089510920D01EDEDF0E08491FF
:100ED0000E940607ECEDF0E084910C940A07369A24
:100EE00008950E942A239093D5018093D4010E94F3
:100EF0007C239093D7018093D6010C945A0C60E028
:100F00008FE10E94E63860E08FE10E94AE3861E038
:100F100081E00E94AE3861E082E00E94AE3861E07C
:100F200083E00E94AE3887E886B90C946307CF93BC
:100F3000DF93D0910D018D2F0E943707882321F078
:100F4000C0913E02C17001C0C0E085E0D89FF001B1
:100F50001124E452FF4F8491C11109C020915D0317
:100F600030915E03232B21F0873011F4C1E085E03E
:100F70000E940A07E0910D01EF5F85E0E89FF00114
:100F80001124E352FF4F84910E9406078CE390E006
:100F90000E9473380E946F073699FECFD0910D01E1
:100FA0008D2F8F5F0E944F0785E0D89FF00111249D
:100FB000E352FF4F84910E9406078CE390E00E9469
:100FC00073380E946F073699FECFC11104C080911B
:100FD0000D010E944F0780910D018F5F0E94430712
:100FE00081110E94840680910D018E5F803118F47A
:100FF00080930D0102C010920D010E945D088823AC
:1010000041F080910D01811104C0DF91CF910C94CA
:101010007107DF91CF9108950C946307CF93DF930D
:101020000E944D0AC0912401D091250102C00E9466
:1010300097078091240190912501C817D907B9F32A
:10104000DF91CF910895CF92DF92EF92FF92CF93ED
:10105000DF93EC010E9430296B017C01CC0EDD1E78
:10106000E11CF11C0E9497070E9430296C157D0538
:101070008E059F05B8F3DF91CF91FF90EF90DF9041
:10108000CF900895E82FF0E0EE0FFF1FE852FE4FDB
:10109000808191810895E82FF0E0EE0FFF1FE25963
:1010A000FE4F808191810895E82FF0E0EE0FFF1F41
:1010B000EA54FE4F80819181089580914002089505
:1010C00080912401909125010895E82FF0E0EE0F22
:1010D000FF1FEA5DFE4F808191810895262F6131C7
:1010E00010F4423040F021E030E0FC0133832283F1
:1010F000318320830895642F70E0F2E02F9F600D0C
:10110000711D1124660F771F660F771F6E5F7F4F6B
:1011100044E050E00C94083A282FCA01213190F4A1
:10112000623080F470E032E0239F600D711D112465
:10113000660F771F660F771F6E5F7F4F44E050E0AA
:101140000C94263A0895FF920F931F93CF93DF9349
:1011500000D000D0CDB7DEB7F12C88E0F89E80013A
:101160001124F801EC5AFF4F459155916591749106
:1011700049835A836B837C83AE014F5F5F4F60E08E
:101180008F2D0E948C08F801E85AFF4F4591559128
:101190006591749149835A836B837C83AE014F5F61
:1011A0005F4F61E08F2D0E948C08F39481E1F8126B
:1011B000D4CF0F900F900F900F90DF91CF911F9190
:1011C0000F91FF900895E82FF0E0EE0FFF1FE25916
:1011D000FE4F20813181E82FE250E53170F4F0E0DC
:1011E000E359FF4F8081882319F0813061F405C0F5
:1011F00081E02333310540F404C081E0293E3340CF
:1012000018F480E0089581E00895CF93C0E08C2F1A
:10121000825E0E94E308882319F0CF5FC630B9F7D9
:101220008C2FCF91089520919A0130919B0180914C
:101230000E0190910F01A0911001B0911101820F48
:10124000931FA11DB11D80930E0190930F01A093D8
:101250001001B0931101089560910E0170910F017A
:1012600080911001909111012DE730E040E050E0B5
:101270000E9494397727652F542F432FCA01089570
:10128000E4E9F1E080819181089580914C01909191
:101290004D01039750F080915201909153010397B3
:1012A00020F083E090E00C94170E80E0089590E029
:1012B000880F991FFC01E259FE4F2081318162178E
:1012C000730718F4261B370B04C0AB01421B530BEA
:1012D0009A01FC01EA5DFE4F2730310518F01182BA
:1012E000108206C0208131812F5F3F4F31832083E0
:1012F000FC01E259FE4F718360830895CF92DF9223
:10130000EF92FF920F931F93CF93DF93C0916E01E3
:10131000D0916F0160917E0170917F018091800179
:10132000909181016817790728F49C01261B370BDF
:10133000B90102C0681B790B8EE10E9457096091C8
:1013400080017091810180918201909183016817E1
:10135000790728F49C01261B370BB90102C0681BD2
:10136000790B8FE10E94570960918401709185018A
:1013700080E20E945709609186017091870181E2A5
:101380000E945709609188017091890182E20E9450
:10139000570960918A0170918B0183E20E9457097D
:1013A0000E940509082F80E0E12CF12C0CC0E82FE9
:1013B000E25EF0E0EE0FFF1FE259FE4F2081318127
:1013C000E20EF31E8F5F8013F2CFB70182E10E941D
:1013D0005709E114F10449F0EC16FD0648F49E01AA
:1013E0002E193F09293E334018F010E000E002C0FA
:1013F000E70112E1BE0183E10E945709602F70E00E
:1014000085E10E945709612F70E084E10E9457092D
:101410000E942C098C010E946D23882329F0E09002
:101420007401F09075010BC00E941B23882329F0E2
:10143000E0907201F090730102C0E12CF12CB70131
:1014400086E10E945709B80188E10E945709970177
:10145000DE010E94463930E1C32E37E2D32EE12C63
:10146000F12CA70196010E949439B90187E10E94ED
:1014700057099801DE010E944639A70196010E9492
:101480009439B90189E1DF91CF911F910F91FF90BC
:10149000EF90DF90CF900C94570910923F0210927A
:1014A0003E0280E094E0899FF0011124E650FE4F57
:1014B00010821182128213828F5F813199F7089511
:1014C000109221011092200110921C0110921D0116
:1014D00010921E0110921F01109218011092190112
:1014E00010921A0110921B011092230110922201F6
:1014F00010921701109216010E9430296093120178
:10150000709313018093140190931501089580E066
:10151000E82FF0E0EE0FFF1FEA5DFE4F1182108210
:101520008F5F8432A9F708950E944D0A0C94870AB0
:10153000109225011092240110920E0110920F01B9
:1015400010921001109211010E940C080E94940A3E
:101550000E94600A80E0E82FF0E0EE0FFF1FE259E2
:10156000FE4F118210828F5F8432A9F70895809117
:10157000400281110AC081E00E94D3040E94980AAF
:1015800081E0809340020C940E080895109240026E
:1015900080E00C94D3042091B8013091B90180917E
:1015A000B6019091B7018217930718F4281B390BE5
:1015B00002C020E030E081E0293E334008F480E0C2
:1015C00008958F929F92AF92BF92CF92DF92EF9247
:1015D000FF92CF93DF93CDB7DEB728970FB6F8947D
:1015E000DEBF0FBECDBFF82E5B0140E0682FCE01FD
:1015F00005960E946E0841E06F2DCE0101960E9473
:101600006E082B813C8140E050E0CF80D884E12CF3
:10161000F12C2C193D094E095F09B50180E090E0DD
:101620008D809E80A12CB12C681979098A099B09AB
:101630000E94643929813A8140E050E02819390933
:101640004A095B090E94B6392C0D3D1D4E1D5F1DD8
:1016500057FF03C020E030E0A901C90128960FB66A
:10166000F894DEBF0FBECDBFDF91CF91FF90EF901A
:10167000DF90CF90BF90AF909F908F9008951F9371
:10168000CF93DF938091240190912501019690934F
:1016900025018093240110E0C12FD0E0DE01AA0FC4
:1016A000BB1FAA0FBB1FA650BE4F20913E02309118
:1016B0003F0240E050E06D917D918D919C910E94A0
:1016C0009439FE01EE0FFF1FE852FE4F3183208355
:1016D000B901812F0E94E10ABC01812F0E945709A4
:1016E0001F5F1131C9F60E947E090E94A934DF9163
:1016F000CF911F910C944D0A0F931F93CF93DF93BB
:10170000C1E0209196013091970180911C01909148
:101710001D01A0911E01B0911F012231310531F050
:10172000C0E02091B6013091B70104C0209194012E
:1017300030919501820F931FA11DB11D80931C0153
:1017400090931D01A0931E01B0931F012091C4012D
:101750003091C5018091180190911901A0911A0151
:10176000B0911B01820F931FA11DB11D8093180121
:1017700090931901A0931A01B0931B01809120014D
:1017800090912101019690932101809320010E9464
:101790003029009112011091130120911401309110
:1017A0001501601B710B820B930B61367A4E81051C
:1017B000910508F47AC0809122019091230101964D
:1017C00090932301809322012091200130912101E7
:1017D00040E050E060911C0170911D0180911E015C
:1017E00090911F010E94943910921C0110921D01CA
:1017F00010921E0110921F01C11106C0B90180E0B4
:101800000E94E10A8C0101C08901C091A401D0911C
:10181000A5010C171D0720F0B8018BE10E945709A4
:10182000B8016C1B7D0B8AE10E94570920912001B1
:101830003091210140E050E0609118017091190150
:1018400080911A0190911B010E9494391092180105
:101850001092190110921A0110921B01B90187E030
:101860000E94E10A2091160130911701909317010F
:1018700080931601BC01621B730B8CE10E94570917
:1018800060912001709121018DE10E945709109211
:101890002101109220010E9430296093120170935F
:1018A00013018093140190931501DF91CF911F9143
:1018B0000F91089540E0A42FB0E0FD01EE0FFF1F4F
:1018C000EE0FFF1FE650FE4FAA0FBB1FAA54BE4FDC
:1018D0002D913C9180819181A281B381820F931FD0
:1018E000A11DB11D80839183A283B3834F5F4131DA
:1018F00011F780913E0290913F02019690933F0232
:1019000080933E020E947C0B80913E0290913F02A8
:101910008436910511F40C943F0B08958F929F9299
:10192000AF92BF92CF92DF92EF92FF92CF93DF936D
:10193000CDB7DEB728970FB6F894DEBF0FBECDBF88
:10194000F82E5B0140E0682FCE0105960E946E08DC
:1019500041E06F2DCE0101960E946E0829813A81E7
:1019600040E050E0CD80DE80E12CF12C2C193D09C7
:101970004E095F09B50180E090E08F809884A12C2A
:10198000B12C681979098A099B090E9464392B8155
:101990003C8140E050E0281939094A095B090E945E
:1019A000B6392C0D3D1D4E1D5F1D57FF03C020E0B5
:1019B00030E0A901C90128960FB6F894DEBF0FBE2A
:1019C000CDBFDF91CF91FF90EF90DF90CF90BF9090
:1019D000AF909F908F9008950C94980A462FE82F0F
:1019E000F0E0EE0FFF1FE259FE4F2081318182505F
:1019F000853130F4E82FF0E0E359FF4F608101C0FA
:101A000061E0C9010C945715825E0C944B088091DB
:101A10006702089580916502811112C00E945D08DD
:101A2000882381F00E946008209141023091420297
:101A3000821B930B9C0181E02530310520F002C010
:101A400081E0089580E008950F931F93CF93DF9373
:101A500010E0CFEFDFEF00E009C0812F0E94040DFE
:101A60008C179D0710F4EC01012F1F5F8091670216
:101A7000181798F3802FDF91CF911F910F91089540
:101A8000CF93DF9390916502911104C0DF91CF91C4
:101A90000C94040D90914B02C82FD0E0992391F043
:101AA0000E94040DCC0FDD1FFE01E45BFD4FC85A00
:101AB000DD4F2081318148815981241B350B280F4E
:101AC000391F07C0FE01EE0FFF1FE45BFD4F2081B1
:101AD0003181C901DF91CF910895CF93C82F8091B3
:101AE0006502882341F0C11106C00E9460089093EE
:101AF000420280934102C09365020E9430296093A4
:101B000043027093440280934502909346020E94E0
:101B1000870A80916402811104C08C2FCF910C94AC
:101B20000F05CF91089580E00E946D0D81E08093B4
:101B3000640208950E94930D80E00C949104EF924A
:101B4000FF920F931F93CF93DF9381E00E94910444
:101B500085E10E944B088093670208E512E03CE4AF
:101B6000E32E32E0F32EC0E0D0E00CC08C2F0E94B8
:101B7000040DF801819391938F01F7018193919363
:101B80007F0121968091670290E0C817D90774F30E
:101B9000109265021092640280E00E946D0D109216
:101BA000420210924102109243021092440210929B
:101BB000450210924602DF91CF911F910F91FF9045
:101BC000EF900895FF920F931F93CF93DF9380912F
:101BD00066020E94400DEC01F12C01E010E01CC0F7
:101BE0008F2D0E94400DAC0180916502802321F071
:101BF000C417D50778F40DC020915B0330915C03C6
:101C00002F5F3F4F369527952C0F3D1F2417350723
:101C100008F4102B000FF39480916702F81600F37C
:101C2000812FDF91CF911F910F91FF9008951F9306
:101C3000CF93DF93EC0110E008C0812F825E0E94F9
:101C400065088C179D0738F01F5F80916702181791
:101C5000A0F381E001C080E0DF91CF911F91089552
:101C6000BF92CF92DF92EF92FF920F931F93CF9389
:101C7000DF938AE090E00E94170E882309F461C088
:101C80000E94240D809366020E94040D8C0162E084
:101C900086E792E00E942E190817190750F17CE49C
:101CA000E72E72E0F72EE8E5CE2EE2E0DE2EC0E071
:101CB000D0E0BB24B39416C08C2F0E94040DF70112
:101CC000819391937F01F601819391936F01801B22
:101CD000910B20915B0330915C032817390708F4BE
:101CE000B12C21968091670290E0C817D90724F3A0
:101CF00002C0BB24B39410924B020E94302960931F
:101D00004702709348028093490290934A02BB2095
:101D100059F0DF91CF911F910F91FF90EF90DF90DD
:101D2000CF90BF900C94930D0E94E20DDF91CF9164
:101D30001F910F91FF90EF90DF90CF90BF900C9488
:101D40006D0DDF91CF911F910F91FF90EF90DF907C
:101D5000CF90BF900895CF9380914B02811119C00D
:101D600081E080934B02809166020E94040DC0E0E6
:101D70000CC08C2F0E94040DEC2FF0E0EE0FFF1F23
:101D8000E85AFD4F91838083CF5F80916702C81727
:101D900080F3CF9108950F931F930E9430290091F3
:101DA0004702109148022091490230914A02601B7B
:101DB000710B820B930B28EE33E040E050E00E9461
:101DC0009439C9011F910F91089583E090E00E941A
:101DD000170E8823C9F080916502811103C00E940B
:101DE000300E12C00E94AB0E0E94E20D90E0809572
:101DF00090952091650230E082239323892B81F412
:101E00000E94CB0E4F9760F40E940A0D882311F0B8
:101E100082E00895809164028823D1F381E00895DF
:101E200080E00E946D0DF0CF1F93CF93DF93EC0104
:101E300010E00FC0812F0E94040D8C179D0710F039
:101E400081E00CC0812F0E94400D8C179D07C0F7C8
:101E50001F5F80916702181768F380E0DF91CF91D0
:101E60001F9108951F93CF93DF93EC0110E00FC0F3
:101E7000812F0E94040DC817D90710F081E00CC013
:101E8000812F0E94400DC817D907C0F71F5F8091AE
:101E90006702181768F380E0DF91CF911F910895D2
:101EA00060916702662321F070E00E94803902C0D1
:101EB00060E070E0CB0108950E94D6110E945F1F80
:101EC00085E00E9412320E942B2A88E00C94123284
:101ED0000E94D6110E94631F86E00E9412320E9467
:101EE0002B2A88E00C941232E0916802F09169028A
:101EF00085919491FC010994E0916802F091690246
:101F0000329685919491FC010994E0916802F091D8
:101F10006902349685919491FC010994CF93DF93E3
:101F20001F92CDB7DEB7811107C00E94401E0E94EC
:101F30007C0F0E94680F0FC0813059F469830E94A2
:101F4000401E0E947C0F6981611105C00E945C0FD8
:101F500002C081E001C080E00F90DF91CF91089531
:101F6000BF92CF92DF92EF92FF920F931F93CF9386
:101F7000DF938C01C62E0E94740F0E94221E0E94C5
:101F8000502A0E94D611F12C82E0D82EC0E0D0E079
:101F9000EE24E3940E94F731811106C0F801EF0DA1
:101FA000F11D84910E9431200E946011B82E84E0BE
:101FB000B81209C0EF2DF0E03196E00FF11FE49167
:101FC000E11123C005C082E0B81202C0F110FA94FA
:101FD000EE2081F00E945A2AD82E6C2D0E948E0F7E
:101FE000E82E882339F00E946008C817D90779F4D1
:101FF000E11003C0C11016C0E12C81E0B812CACFB5
:102000000E94401E0E947C0F0DC0F394E1CF0E94FD
:102010006008EC010E94850FD82E6C2D0E948E0F57
:10202000E82EE6CF8D2DDF91CF911F910F91FF907C
:10203000EF90DF90CF90BF900895FC012481205253
:10204000621710F40C947717862F90E0821B910989
:102050000E94F4196EE00C94141360E08AE692E09A
:102060000E94751887FD0AC0811102C00C94542F7C
:10207000992787FD909501970C94352508950E9426
:10208000D8040E9404330E94A02F62E471E082E32E
:1020900091E00E94421F88EE93E00E94230880E0B6
:1020A0000C94863760E571E08AE692E00E9486171C
:1020B00086E890E090936B0280936A02EEE6F2E08D
:1020C0008081805E80830895CF93DF93EC010E942E
:1020D000CE118B819C810E9411130E94D2116A81C2
:1020E00088819981DF91CF910C94AD12FC01878199
:1020F0008F3118F48F5F8783089586818F5F868381
:102100000895FC018781882319F081508783089501
:1021100086818150868308951F93CF93DF93FC01BE
:10212000C681D0E06D2F80E00E94C8111C2F105F87
:102130008C2FCF5F0E946B138C2FC113FACFDF5F00
:10214000D23081F7DF91CF911F9108951F93CF93E4
:10215000DF93EC0188EE90E00E944F161FEF8E8116
:10216000181721F0CE010E948C101E818F81682FDC
:1021700070E094E0759567959A95E1F78F700E94ED
:10218000C8110E946011823049F0843019F081300A
:1021900049F413C0CE010E947610E1CFCE010E9417
:1021A0008110DDCF8830D9F68D81E881F981E80F83
:1021B000F11D8F819E81890F8083DF91CF911F91C7
:1021C0000895FC01718360834283348323831582E5
:1021D00080E2868317820895CF93DF93EC0188EE27
:1021E00090E00E944F160E94D611CE010E9464100A
:1021F00061E08D810E94C8110E9460118230B1F0AF
:10220000843041F08130C1F488EE90E00E9457168E
:1022100080E026C04D81242F30E08A8190E0019734
:10222000281739072CF74F5F4D83E2CF8D81882324
:10223000F9F281508D83DCCF8830D1F682E00E94A4
:10224000B711823048F083E00E94123288EE90E0AD
:102250000E94571681E004C0CE010E94A610C3CF91
:10226000DF91CF9108950C946C04E0917402F0E03A
:10227000EE0FFF1FE45AFE4F25913491C9010895D6
:10228000CF93DF93D82F0E946C0407C082E390E0C5
:102290000E9423080E946C04DC2FC82F8D13F6CFF8
:1022A000109274021092730280937502882319F0C1
:1022B00080E00E941E3280917502DF91CF910895D7
:1022C000EF92FF920F931F93CF93DF93C0E0D0E084
:1022D000F12C0AEF10E016C00E946C04F82E81E089
:1022E00090E00E94230880917502F81202C02196A6
:1022F00009C08F2DDF91CF911F910F91FF90EF902B
:102300000C944011E09074022E2D30E0220F331F08
:10231000F901E659FE4F65917491C8010E94803918
:102320006F5F7F4FC617D707B8F2FF20B9F0409113
:1023300073024F5F40937302F901E858FE4F859195
:102340009491242F30E02817390740F085E08E154E
:1023500018F0E394E0927402109273028091750277
:10236000DF91CF911F910F91FF90EF900895CF9340
:10237000DF93D82FC09175020E9460119091740272
:102380009D1711F08C17C1F3892FDF91CF9108951C
:10239000462F682F88EE90E00C94661660E080E08F
:1023A0000C94C81161E080E00C94C81188EE90E0B4
:1023B0000C949616CF93DF93FC01DB018C9188235C
:1023C00089F0C081D1814883808191810196918378
:1023D00080838C9181508C93882321F00190F0812F
:1023E000E02D1082DF91CF910895BF92CF92DF92BE
:1023F000EF92FF920F931F93CF93DF93EC018B012A
:102400007A014115510501F1CA010E94E139F80133
:102410009081B82E981708F4B92ECB2CD12CA60198
:10242000B701888199810E94EA39288139812C0D70
:102430003D1D39832883F80180818B19808388238F
:1024400019F0E881F9811082DF91CF911F910F91EE
:10245000FF90EF90DF90CF90BF900895EF92FF92A2
:102460001F93CF93DF9300D000D0CDB7DEB77C01B0
:10247000CA014B835C8369837A830E94AC29182F3D
:1024800069817A81DB018C914B815C81811768F4D1
:102490004FE3C7010F900F900F900F90DF91CF91F6
:1024A0001F91FF90EF900C94DA11F7012081318198
:1024B000210F311D31832083DB018C91811B8C9393
:1024C000882321F00190F081E02D1082F9012AE0AB
:1024D00030E00CC0CA01B9010E948039405DBAE009
:1024E0006B9F4019112442931150AB011111F2CF8F
:1024F0000F900F900F900F90DF91CF911F91FF9051
:10250000EF9008950F931F93CF93DF93CDB7DEB76E
:102510002B970FB6F894DEBF0FBECDBF8E010F5FB5
:102520001F4F1A87098727E02B87AC01BE01655F23
:102530007F4FCE0109960E942E12B80188EE90E0DE
:102540000E941D382B960FB6F894DEBF0FBECDBF8C
:10255000DF91CF911F910F9108951F93CF93DF9338
:10256000CDB7DEB761970FB6F894DEBF0FBECDBF13
:102570000097D1F0162F613108F010E1412F50E0A3
:10258000BC01CE0101960E94F939E1E0F0E0EC0FC8
:10259000FD1FE10FF11D1082BE016F5F7F4F88EEBE
:1025A00090E00E941D3801C080E061960FB6F8945B
:1025B000DEBF0FBECDBFDF91CF911F9108951F9356
:1025C000CF93DF93CDB7DEB761970FB6F894DEBF38
:1025D0000FBECDBF0097D1F0162F613108F010E18A
:1025E000412F50E0BC01CE0101960E94EA39E1E0A2
:1025F000F0E0EC0FFD1FE10FF11D1082BE016F5FD7
:102600007F4F88EE90E00E941D3801C080E0619607
:102610000FB6F894DEBF0FBECDBFDF91CF911F91F3
:10262000089560E10C94DF12CF92DF92EF92FF9257
:102630000F931F93CF93DF93CDB7DEB762970FB69B
:10264000F894DEBF0FBECDBF009761F1613108F095
:1026500060E17C01CC24C394D12CCC0EDD1E86011C
:102660001CC0C7016A8B0E94183AF80181938F0140
:10267000FFEFEF1AFF0A6A8981110FC0E1E0F0E075
:10268000EC0FFD1FE60FF11D1082BE016F5F7F4F43
:1026900088EE90E00E941D3806C0802F8C198617A6
:1026A00000F3ECCF80E062960FB6F894DEBF0FBE69
:1026B000CDBFDF91CF911F910F91FF90EF90DF90F1
:1026C000CF900895882319F08AE891E002C08EE83F
:1026D00091E00C941113682F88EE90E00C941F3851
:1026E000CF93DF931F92CDB7DEB7682F06C080E28D
:1026F00069830E946B13698161506430C4F786E876
:1027000091E00F90DF91CF910C94DF12CF93DF9384
:10271000D82FC0E004C080E20E946B13CF5FCD13BE
:10272000FACF8C2FDF91CF91089580E10C9486131E
:102730006AE00E947439892F805D0C946B13DF92DC
:10274000EF92FF920F931F93CF93DF93EC01162F1D
:1027500016160CF059C064E670E00E948039D62E3F
:10276000E72ECB010E94AC29082F23E0F22EF80EB1
:1027700004C080E20E946B131150F116D4F3412F74
:10278000552747FD50952F2D332727FD3095235092
:1027900031094217530754F4812FDF91CF911F91D4
:1027A0000F91FF90EF90DF900C9470138D2D9E2D64
:1027B0000E948212CE0164E670E00E948039EC0132
:1027C000101B012F015011161CF48EE20E946B1396
:1027D000102F1150101644F4CE016AE070E00E94F0
:1027E0008039862F0E949813111674F4CE016AE086
:1027F00070E00E948039DF91CF911F910F91FF907F
:10280000EF90DF900C949813DF91CF911F910F916F
:10281000FF90EF90DF900895CF92DF92EF92FF92BA
:102820000F931F93CF93DF93EC01162FC42E161630
:102830000CF088C068EE73E00E948039D62EE72E37
:10284000CB010E94AC29F82E082F0C5F04C080E257
:102850000E946B1311500117D4F31017DCF0C11054
:1028600019C0CE010E94AC29082F03C080E20E944B
:102870006B1311500117D4F3CE010E9482128DE622
:10288000DF91CF911F910F91FF90EF90DF90CF904C
:102890000C946B13412F552747FD5095202F33275C
:1028A00027FD309524503109421753075CF4812FDE
:1028B000DF91CF911F910F91FF90EF90DF90CF901C
:1028C0000C9470138D2D9E2D0E948212CE0168EE05
:1028D00073E00E948039EC011F19012F015011167D
:1028E0001CF48EE20E946B13102F1150101644F44A
:1028F000CE0164E670E00E948039862F0E94981312
:10290000CE0164E670E00E948039EC01012F015095
:1029100011163CF46AE070E00E948039862F0E9414
:10292000981310167CF4CE016AE070E00E948039A2
:10293000DF91CF911F910F91FF90EF90DF90CF909B
:102940000C949813DF91CF911F910F91FF90EF900E
:10295000DF90CF9008956F927F928F929F92AF9267
:10296000BF92CF92DF92EF92FF920F931F93CF937C
:10297000DF937C01962E742E822E16160CF044C026
:1029800021119A94C7010E94AC29C0E0D0E0082F21
:1029900010E0A92CBB24A7FCB09404C0872D0E9492
:1029A0006B132196692C6C1A6501CC1ADD0A0C1583
:1029B0001D05A4F3882019F08DE20E946B13C01648
:1029C000D1068CF4862DDF91CF911F910F91FF904E
:1029D000EF90DF90CF90BF90AF909F908F907F90BF
:1029E0006F900C947013C701DF91CF911F910F91DD
:1029F000FF90EF90DF90CF90BF90AF909F908F901F
:102A00007F906F900C948212DF91CF911F910F9164
:102A1000FF90EF90DF90CF90BF90AF909F908F90FE
:102A20007F906F90089520E00C94AB1440E20C94DA
:102A30001315CF93DF936CE370E00E9480399B0104
:102A4000EC0140E363E0C9010E9413158AE30E9490
:102A50006B1340E362E0CE01DF91CF910C9413152C
:102A6000292F221F2227221F19F091958195910964
:102A700040E20C94AB14161634F461500E949F137C
:102A800083E40C946B130895161634F461500E947D
:102A9000161585E20C946B13089563303CF0625078
:102AA0000E94161582E991E00C9411130895CF93BA
:102AB000DF93C62F14167CF5642F6150C23071F07D
:102AC00028F4CC23B9F0C130C1F406C0C43059F0A9
:102AD00080F0C53091F409C0D6E510C0642FDF91B5
:102AE000CF910C943B15D4EF06C00E94301585E5BC
:102AF0000EC06150D1E440E002C0D5E541E00E9443
:102B00000C148D2F0E946B13C33029F488E6DF91DB
:102B1000CF910C946B13DF91CF910895462F64E011
:102B20000C945715462F61E00C945715462F60E022
:102B30000C945715462F63E00C945715CF93DF93F1
:102B4000EC0160E08E810E94E63881E090E00E9416
:102B5000733861E08E810E94E63881E090E00E9447
:102B6000733860E08E810E94E63884E690E0DF9161
:102B7000CF910C947338CF92DF92EF92FF920F9324
:102B80001F93CF93DF937C01C0E0D0E0C62ED12C01
:102B900087010C0F1D1F61E0F80187810E94AE388C
:102BA000B6010C2E02C0759567950A94E2F7617024
:102BB0007727F80187810E94E6382196C430D10535
:102BC00039F7C701DF91CF911F910F91FF90EF90DF
:102BD000DF90CF900C949E15CF92DF92EF92FF92F0
:102BE0000F931F93CF93DF937C01C0E0D0E0C62EFC
:102BF000D12C87010C0F1D1F61E0F80187810E9415
:102C0000AE38B6010C2E02C0759567950A94E2F7AE
:102C100061707727F80187810E94E6382196C830D5
:102C2000D10539F7C701DF91CF911F910F91FF9027
:102C3000EF90DF90CF900C949E151F93CF93DF936E
:102C4000EC01162F642F8C810E94E6388D818F3F16
:102C500019F060E00E94E6388F85612F84FF06C07E
:102C6000CE01DF91CF911F910C94EC1570E084E0C0
:102C7000759567958A95E1F7CE010E94BB15612F86
:102C8000CE01DF91CF911F910C94BB1541E00E94C2
:102C90001D1681E090E0089540E00C941D16FC01A3
:102CA0006089262F2160208B69600C944C16FC01F2
:102CB00060896E7F608B68600C944C16FC016089A3
:102CC000262F2460208B6C600C944C16CF93DF93DE
:102CD000CDB7DEB728970FB6F894DEBF0FBECDBFD5
:102CE00028E0E5E6F0E0DE01119601900D922A95CC
:102CF000E1F7FC012389421710F0422F4150E1E037
:102D0000F0E0EC0FFD1F22E0429FE00DF11D1124C9
:102D10002081260F2068622F28960FB6F894DEBF18
:102D20000FBECDBFDF91CF910C944C1661E00E9495
:102D30004C1680ED97E00C947338CF93DF93EC0141
:102D4000423018F08F8588608F874B8B1C8A222336
:102D500029F0413019F48F8584608F8780E593ECEA
:102D60000E94733860E08C810E94E63860E08E81BA
:102D70000E94E6388D818F3F19F060E00E94E638AE
:102D80006F8564FD1DC063E0CE010E94BB1584E920
:102D900091E10E94733863E0CE010E94BB1584E983
:102DA00091E10E94733863E0CE010E94BB1586E971
:102DB00090E00E94733862E0CE010E94BB1516C0FD
:102DC0006062CE010E944C1684E991E10E94733842
:102DD0006F856062CE010E944C1686E990E00E94E9
:102DE00073386F856062CE010E944C166F856062F9
:102DF000CE010E944C1684E0888BCE010E945E16A4
:102E0000CE010E94961682E0898B66E0CE01DF91AA
:102E1000CF910C944C166F927F928F92AF92CF927B
:102E2000EF920F931F93CF93DF93CDB7DEB73C01A3
:102E3000162F842F5D854E853F859889F301848305
:102E400025830683E782C086A186828653874487CE
:102E50003587968761E00E94AE38F30185818F3F08
:102E600019F061E00E94AE3861E0F30186810E94B2
:102E7000AE38112319F0F301178603C080E1F30186
:102E8000878720E041E060E1C301DF91CF911F918E
:102E90000F91EF90CF90AF908F907F906F900C94A8
:102EA0009D168F92AF92CF92EF920F93DC01139603
:102EB0001C921E921297ECE8F0E0ED93FC931F92A7
:102EC0001F921F921F928C2CAE2CC02EE22E042F2C
:102ED0002FEF462F61E00E940B170F900F900F907D
:102EE0000F900F91EF90CF90AF908F900895DC01ED
:102EF0001796ED91FC911897B2E06B9FE00DF11DD4
:102F0000112425913491C9010C9411130F931F932F
:102F1000CF93DF93EC018B01CB010E946329682FD3
:102F2000CE010E94E91784E990E09983888318878D
:102F30000F83DF91CF911F910F910895DF92EF9250
:102F4000FF920F931F93CF93DF93EC01F62E6987C7
:102F50001A8681E08D8382E0D82EEE24E3948E01E0
:102F6000075F1F4F0E946011482F823011F084309C
:102F700061F4E881F9810280F381E02D6F2DCE01AB
:102F80000995F986DA86ED8204C0813089F08830AF
:102F900079F0C8010E943F2A8111ED828D8188233A
:102FA00019F0CE010E9417188A858F5F8A87DACFC1
:102FB0008FEF898781E08E838D83483009F080E030
:102FC000DF91CF911F910F91FF90EF90DF900895C7
:102FD0000895FC018AE990E0918380831282138234
:102FE000648381E0858386830895FC018281811159
:102FF00003C081E082830895438190E0840F911D96
:10300000248130E0215031098217930714F44F5F77
:1030100043830895FC018281882319F081508283C3
:1030200008958381882311F08150838308951F932D
:10303000CF93DF93EC0110E0612F80E00E94C81174
:1030400080E20E946B13E881F9816B81610F01902E
:10305000F081E02DCE0109950E9495131F5F12307B
:1030600059F76A8180E00E94C8118EE30E946B13B9
:103070006A818FE00E94C8118CE30E946B131D824D
:10308000DF91CF911F9108950F931F93CF93DF93FB
:10309000EC010E946011182F0E94F731882321F063
:1030A00081E08D831FE71BC00B818A81080F1230DE
:1030B00031F0143039F4CE010E94F51703C0CE016F
:1030C0000E940A188B819A81890F081711F081E0FC
:1030D0008D838D81882319F0CE010E941718812FCE
:1030E000DF91CF911F910F910895EF92FF921F935F
:1030F000CF93DF931F92CDB7DEB77C0181E0F7015C
:10310000858311E0C70169830E9444186981811198
:1031100002C0F7011682F7019681911108C088302C
:1031200031F481E0868383819281890F09C066230F
:1031300011F0F7011583813029F79111E3CF8FEF5B
:103140000F90DF91CF911F91FF90EF9008950F9313
:103150001F93CF93DF93EC018B0150E00E942E125E
:103160004AE3B801CE01DF91CF911F910F910C94EA
:10317000DA11EF92FF920F931F93CF93DF9300D05A
:103180001F92CDB7DEB78C01462F09969A838983AB
:103190008EE08B83D801EC91F0E0EE0FFF1FEB5631
:1031A000FE4FE590F490BE016D5F7F4FCE0101961A
:1031B0000E94A718A701BE016D5F7F4FCE01019647
:1031C0000E94F51140E2BE016D5F7F4FCE01019676
:1031D0000E94DA11F80141815281BE016D5F7F4F7B
:1031E000CE0101960E942E124FE2BE016D5F7F4F0D
:1031F000CE0101960E94DA11D80117964D915C918B
:103200001897BE016D5F7F4FCE0101960E942E126E
:103210000F900F900F90DF91CF911F910F91FF9022
:10322000EF90089527E1289FB001299F700D112488
:1032300064577F4F47E150E086E792E00C94083AEC
:1032400027E1289FB001299F700D112464577F4FFB
:1032500047E150E086E792E00C94263ADC01EC91DD
:10326000B5E0EB9FF0011124E60FF11DEE0FFF1FFB
:10327000EB55FE4F25913491C9010895CF93DF930B
:10328000EC010E942E194F815885849F9001859FE3
:10329000300D949F300D1124C901DF91CF91089515
:1032A0000F931F93FC01A181B281209155033091AE
:1032B00056030E94463924E630E040E050E00E9488
:1032C000943989019A01093EFDEF1F072105310557
:1032D00020F008EE1DEF20E030E0C8011F910F91B3
:1032E0000895FC012081213029F42091510330916F
:1032F000520309C0223029F420914F03309150032A
:1033000002C020E030E0FC0187819085289FA00169
:10331000299F500D389F500D1124CA010895EDE4E6
:10332000F3E0808191810895FC016081F9E06F9F55
:10333000B00111246B507E4F49E050E00C94D83915
:10334000DC01EC91F0E0EE0FFF1FEB56FE4F2591F4
:103350003491C9010C94DF1260E170E00C94A01963
:10336000CF93DF93EC01888160E0811108C0CE012A
:103370000E943E1967E00E94921587E011C0CE01BD
:103380000E943E1965E00E9492158FE20E946B1325
:103390008F8198850E94821283E40E946B1388E0DB
:1033A000DF91CF91089566E0FC01838194810E94B2
:1033B000961586E0089566E0FC01858196810E945D
:1033C000961586E00895FC0181819281883EFDEF8B
:1033D0009F0729F48DE392E00E94111303C067E078
:1033E0000E949A1588E0089547E1489F9001499FFF
:1033F000300D11242B563F4FC90108950F931F9391
:10340000CF93DF93CDB7DEB7A4970FB6F894DEBFA6
:103410000FBECDBF8C01AB01BC01CE0101960E9455
:10342000AB1BCE0101960E94191C87E1FE013C9660
:10343000D80101900D928A95E1F7A4960FB6F89401
:10344000DEBF0FBECDBFDF91CF911F910F910895C9
:10345000FC012081260F283010F4208302C0FC01DB
:1034600010820C9494190F931F9361E00E943E19EF
:103470009C0140E050E060E870EF8AEF92E00E942B
:10348000943989019A01093883E11807210531052A
:1034900020F008E813E120E030E0C8011F910F910F
:1034A00008950F931F9361E00E943E199C0140E034
:1034B00050E060E47BE48CE490E00E949439890160
:1034C0009A01013D87E018072105310520F000ED44
:1034D00017E020E030E0C8011F910F9108950F938D
:1034E0001F93CF93DF9300D0CDB7DEB78C016983F4
:1034F0007A830E94331AAC0169817A81C8010396EC
:103500000F900F90DF91CF911F910F910C94DC29B8
:103510000F931F93CF93DF9300D0CDB7DEB78C010D
:1035200069837A830E94511AAC0169817A81C8014A
:1035300005960F900F90DF91CF911F910F910C94F2
:10354000DC2961E00E942E19BC0184ED92E60E9404
:103550008039CB0108950F931F93CF93DF9300D051
:10356000CDB7DEB78C0169837A830E94A11AAC01C2
:1035700069817A81C80107960F900F90DF91CF91F2
:103580001F910F910C94DC29CF93DF93EC010E94E3
:10359000A11A2F8138858217930710F498878F839B
:1035A000CE010E94331A2B813C818217930710F4BD
:1035B0009C838B83CE010E94511A2D813E818217FC
:1035C000930710F49E838D83DF91CF910895CF935D
:1035D000DF93EC0148EE5DEF01960E94DC298981C2
:1035E0009A819C838B832881233039F49C01369502
:1035F0002795369527953C832B839E838D83CE011B
:10360000DF91CF910C94C41ADF92EF92FF920F9347
:103610001F93CF93DF9300D01F92CDB7DEB749E061
:1036200050E06BE272E086E792E00E94D83986E7CC
:1036300092E00E94C41A00E010E05EE0D52E6FE731
:10364000E62E62E0F62EDB82FA82E982402F4F5F9F
:10365000BE016D5F7F4FCE0101960E94A718C80181
:103660000E9420190F5F1F4F0032110561F70F9064
:103670000F900F90DF91CF911F910F91FF90EF90DE
:10368000DF90089508950895262F443019F06FEFC4
:103690007FEF02C061E070E0223089F028F422233D
:1036A00041F02130A9F408C0233061F0243081F4C6
:1036B0000CC00B960C94281A0B960C94AB1A0B9614
:1036C0000C94E71A0B960C946F1A0B960C94881AAC
:1036D00008951F93CF93DF93EC01162F0E94771765
:1036E000CE0109960E94342A882311F0298501C051
:1036F0002FEF332727FD3095812F90E028173907CA
:1037000029F11230A9F028F4112341F01130F1F41D
:103710000AC0133091F01430C9F414C0CE010B96D6
:103720000E94AC1913C0CE010B960E94B0190EC0B6
:10373000CE010B960E94E31909C0CE010B960E94A0
:10374000D31904C0CE010B960E94DB1980E0DF91F3
:10375000CF911F910895EF92FF920F931F93CF93F4
:10376000DF93EC018B017A0161E772E00E9486171A
:103770008FEF898780EA90E09983888387E1F80159
:10378000DE011B9601900D928A95E1F7FBA2EAA259
:10379000DF91CF911F910F91FF90EF9008950F93BC
:1037A0001F93CF93DF93CDB7DEB728970FB6F8946A
:1037B000DEBF0FBECDBF8C01BC016C5E7F4F21E828
:1037C00032E04EE050E0CE0101960E94E110CE01C1
:1037D00001960E94EC1081E0F801858328960FB6CF
:1037E000F894DEBF0FBECDBFDF91CF911F910F9137
:1037F0000895CF93DF93EC016AA17BA16F5F7F4FA8
:103800000B960E94B9180E94D6110E94CE118CE826
:1038100092E00E9411130E94D2116EE0CE014496F4
:103820000E94AD120E942B2A83E0DF91CF910C946D
:103830001232DF92EF92FF920F931F93CF93DF9399
:10384000CDB7DEB767970FB6F894DEBF0FBECDBF1A
:103850008C0187E1D82E9BE0E92EF12CE00EF11EC1
:1038600060E0C8010E94751887FD2BC0853019F0F3
:10387000863049F404C0C8010E94F91BF1CFC80189
:103880000E94CF1BEDCFF701DE0111969D2D019017
:103890000D929A95E1F7682FC8010E949E17811139
:1038A00009C0FE013196D7018D2D01900D928A95A8
:1038B000E1F7D6CF83E00E941232C7010E94C41AFA
:1038C000CFCF67960FB6F894DEBF0FBECDBFDF91A6
:1038D000CF911F910F91FF90EF90DF90089580910D
:1038E000490390914A03892BA1F08CE10E944B0877
:1038F00065E02AE0AC01249FC001259F900D1124B2
:103900000E9430158DE60E946B1383E40E946B13B6
:1039100004C08BE693E00E9411130C9495138AE186
:103920000E944B0865E00E9430158DE60E946B13E3
:1039300086E50E946B130C949513CF93DF9300D010
:10394000CDB7DEB789839A830E94CE1189819A818F
:103950000E9411130E94D2118091B2029091B30281
:103960000E94E139892B51F084E593E00E94111304
:103970008091B2029091B3020E9411130F900F90A8
:10398000DF91CF910C94951390E0880F991F62E01E
:1039900088539D4F0C94DF120F931F93CF93DF93A7
:1039A00061E086E792E00E943E198C0162E086E7C2
:1039B00092E00E943E19EC0183E10E944B088017BF
:1039C000910790F4C817D90788F49C012C1B3D0B74
:1039D000C8018C1B9D0B64E670E00E948039C90110
:1039E0000E948039862F03C084E601C080E0DF9109
:1039F000CF911F910F910895613011F40C94400DF7
:103A00000C94D526CF93DF93D82FC62F825E0E94C9
:103A1000E308882351F06C2F8D2F0E94FC1C46E098
:103A20006C2FDF91CF910C94571585EE92E0DF91CA
:103A3000CF910C9411130F931F93CF93DF93C82F43
:103A4000162F0E94CE110E940A0D811108C083E03A
:103A500090E00E94170E882341F080E209C0809117
:103A60004B02882321F082E403C08DE601C082E688
:103A70000E946B13809165028823C9F0D0E001E0B9
:103A800080916602D81731F080916502802321F081
:103A900081E303C08FE501C080E30E946B13000F38
:103AA000DF5FD63069F780E20E946B1303C087E0C6
:103AB0000E948613DC2FDF5F8D2F0E9498138AE30C
:103AC0000E946B13C1112AC00E946D23882331F11B
:103AD0000E947C23892B39F521C00E9495130E94F6
:103AE000D2110C2F0E5F802F0E9498138AE30E9440
:103AF0006B13612F8D2F0E94021D8C2F8D5F0E94F2
:103B000098138AE30E946B13612F802F0E94021D7D
:103B1000DF91CF911F910F910C949513612F8C2FF2
:103B20000E94021DDACF8CEE92E00E941113D5CFD5
:103B300088E10E944B0868E00E949A1580E20C948C
:103B40006B130E94CE1186E792E00E94501968E044
:103B50000E949A1580E20E946B130E94BE2667E0C5
:103B60000E9496150E9495130E94D21181EF92E057
:103B70000E94111367E08091390390913A030E94EB
:103B800092150C9495130F931F9360919802709166
:103B9000990280919A0290919B0220918D0222239A
:103BA00071F00E94302900919802109199022091A1
:103BB0009A0230919B02601B710B820B930B28EED3
:103BC00033E040E050E00E949439C9011F910F9109
:103BD00008950E941B23811110C00E946D23882329
:103BE00031F00E941B2381110AC084E40BC00E94A3
:103BF0000A0D811106C08EE405C083E403C085E48C
:103C000001C082E40E946B1380E20E946B130E9449
:103C1000C31D0E94191580E20C946B130E94CE11F3
:103C20000E94981D67E086E10E94EE0C0E949513A9
:103C30000E94D2110E94E91D67E083E10E94EE0C10
:103C40000C9495130E943029609398027093990206
:103C500080939A0290939B02109294021092950284
:103C60001092960210929702109290021092910276
:103C7000109292021092930281E080938D02089537
:103C80000F931F930E94302900919802109199027E
:103C900020919A0230919B02601B710B820B930B57
:103CA000609398027093990280939A0290939B027A
:103CB00010928D021F910F9108950E94212381116E
:103CC0001DC00E947323811119C00E940A0D882310
:103CD00051F18091940290919502A0919602B09139
:103CE000970280599F4FAF4FBF4F8093940290939C
:103CF0009502A0939602B093970208958091900246
:103D000090919102A0919202B091930280599F4F9D
:103D1000AF4FBF4F8093900290939102A093920275
:103D2000B0939302D2CF0895CF92DF92EF92FF9299
:103D30000E94CE118AEF92E00E9411130E94C31DCF
:103D40000E9419150E94D21185E093E00E94111380
:103D500060919402709195028091960290919702E1
:103D600038EEC32E33E0D32EE12CF12CA7019601BF
:103D70000E949439C9010E94191588E093E00E94BD
:103D80001113609190027091910280919202909132
:103D90009302A70196010E949439C901FF90EF9008
:103DA000DF90CF900C9419150E94CE118BE093E018
:103DB0000E9411130E94DF2668E00E948E150E9467
:103DC00095130E94D21182E10E94E308882349F0F2
:103DD00084E193E00E9411130E94E52668E00E94AE
:103DE0008E150C9495130E94CE118DE193E00E94E4
:103DF000111367E086E00E94EE0C0E9495130E946A
:103E0000D21185E293E00E94111347E061E08091B6
:103E10005703909158030E9457150C9495130E94D4
:103E2000CE118DE293E00E94111367E080E00E94C2
:103E3000EE0C0E9495130E94D21184E393E00E943D
:103E4000111367E082E10E94EE0C0C9495130E941E
:103E5000CE118BE393E00E9411138091490390915E
:103E60004A03892B29F065E087E00E94EE0C04C02C
:103E700081E493E00E9411130E9495130E94D211D5
:103E80000C9495130F931F93CF93DF9300D0CDB76E
:103E9000DEB78B0189839A830E94D6110E94CE11CE
:103EA00089819A810E9411130E94D211C8010F903A
:103EB0000F90DF91CF911F910F910C94111383E418
:103EC00093E00C949D1C8DE593E00C949D1C0E9446
:103ED000CE110E94981D0E946F1C0E94D2110E9458
:103EE000E91D0C948F1C0E94CE1184E793E00E9480
:103EF000111367E08BE10E94EE0C0E9495130E9463
:103F0000D2118DE793E00E9411130C948F1C0E9434
:103F1000CE1187E893E00E9411138091490390919C
:103F20004A03892B41F069E08091160190911701B5
:103F30000E943B1504C08DE893E00E9411130E947B
:103F400095130E94D21186E993E00E9411130C94FC
:103F50006F1C6DEA73E080EA93E00C94421F0E94AC
:103F6000A91F0C942B2A6EEC73E08DEB93E00E945A
:103F7000421F88E893E10C9446290E94CE1189EDF6
:103F800093E00C941113CF930E94CE1164E070E083
:103F900086E792E00E94A01980E20E946B1386E7F8
:103FA00092E00E94B01980E20E946B138091B402EB
:103FB0000E94C41C0E94D2110E94CC1C90E0843646
:103FC000910569F48EE892E00E94342A882321F05A
:103FD00084E00E9486130AC08AEE93E005C062E086
:103FE0000E9416158FEE93E00E9411138EE892E066
:103FF0000E94342A882319F0C0918E0201C0CFEFAD
:10400000C0FF05C065E080E00E94EE0C03C085E0C3
:104010000E94861380E20E946B1380917602845086
:104020008430A8F4C1FF05C065E082E10E94EE0C77
:1040300003C085E00E948613C2FF05C00E940509E7
:10404000CF910C94981380E2CF910C946B1366E09F
:1040500080917702909178020E949A15CF910C94EA
:10406000951390918F029F5F90938F02883049F152
:1040700068F48430E1F030F48230A9F0B0F481309B
:1040800099F524C08630B9F0C0F413C08C3011F11A
:1040900020F48A3039F1E0F417C08E30F9F0E0F006
:1040A0008F3011F51DC00C940E1E0C94A11D0C94A4
:1040B000941E0C94271F61E005C061E083E00C941E
:1040C0001B1D64E080E0FBCF64E0F8CF0C94C31FBD
:1040D0000C94D41E0C940F1F0C94F31E0C94731F9D
:1040E0000C94871F0C94671F08958FEF80938E02A6
:1040F00008950F931F93CF93DF930E944523C091A0
:104100007902D0917A0261E086E792E00E943E193E
:104110008C01CE0165E070E00E9480398FE00E9442
:104120008E0CEC0140E0BC01C8010E9409278FE021
:104130000E941D27CE01DF91CF911F910F910C940A
:104140002F2381E00C9453230E944509882321F0FA
:104150000E942A230C94C527089510929C020C9467
:104160007920CF93DF930E94A4200E944009EC01A4
:1041700080919C02811111C062E086E792E00E946A
:104180003E198C179D0748F481E080939C02809132
:10419000790290917A020E943F230E944509882368
:1041A000D9F164E086E792E00E943E198C179D07E2
:1041B00058F132C080919D02882389F08AE10E94E3
:1041C0004B08EC0186E792E00E947119D195C195E8
:1041D000D1098C179D071CF480E094E017C08091F2
:1041E0009E02811101C00EC08CE10E944B08EC01BF
:1041F00086E792E00E948F198C179D071CF484E0DB
:1042000094E004C082E00FC088EF93E09093B30283
:104210008093B20281E007C0809122019091230136
:10422000029740F6EFCFDF91CF91089580939E02E1
:1042300060939D0208957093A2026093A1029093EF
:10424000A00280939F0208950F931F93CF93DF9353
:10425000C0919F02D091A002CE010E94500F8C010C
:104260000E944009C817D90738F4C801DF91CF91DF
:104270001F910F910C94320F81E0DF91CF911F912C
:104280000F9108950F931F93CF93DF930E942421E2
:10429000182F0E947C23EC010E944509882311F00D
:1042A00001E001C0012F8091A302882329F0BE0103
:1042B000812F0E94752701C0812F882329F081E07A
:1042C0000E94B42381E00DC0011101C009C0BE01EC
:1042D000812F0E9494288C179D0711F00E9498232B
:1042E00082E0DF91CF911F910F9108950E94A62344
:1042F0000E949F0D1092A30280E10C941D2781E083
:104300000E94B4230C949A0DBC0180E10E948E0C93
:104310000C94AC260F931F93CF93DF938C01EB018A
:104320000E941B21BE0180E10E948E0C40E0BC0176
:10433000C8010E940927CE016AE070E00E9480391E
:10434000CB01DF91CF911F910F910C9484210E949A
:104350009F0D0E9445238FE00C941D2781E00E9451
:1043600053230C949A0D0F931F93CF93DF931F92B7
:10437000CDB7DEB78C018FE049830E948E0C498156
:10438000BC01C8010F90DF91CF911F910F910C9448
:104390000927BC018FE00E948E0C0C94AC260F9371
:1043A0001F93CF93DF93C0913903D0913A03CE018D
:1043B0000E94500F8C010E9440098C179D0738F411
:1043C000C801DF91CF911F910F910C94140F81E0E0
:1043D000DF91CF911F910F9108951F93CF93DF939A
:1043E0000E94CF21182F0E942A23EC01BC01812FAB
:1043F0000E947527882329F081E00E94532381E0E1
:104400001BC00E94450981110BC0111109C0CE01CA
:104410000E94C626811104C00EC00E942F230BC02B
:104420000E940A0D811107C0BE01812F0E949428AD
:104430008C179D0791F782E0DF91CF911F9108952E
:104440000E94AE210E947F210C949A0DCF93DF939E
:104450001F92CDB7DEB79091A502913039F018F0D8
:10446000923081F406C00E94ED210CC00E944221CE
:1044700009C00E94E50E823089F089830E942022C3
:1044800089810CC0813051F49091A402992331F0BC
:1044900082E08093A5020E949F0D82E00F90DF9141
:1044A000CF9108950E949F0D8091A6029091A7023E
:1044B0000E94500F0E94320F882329F00E94A721EA
:1044C0001092A50208950E94762181E08093A302B4
:1044D0008093A50208958093A40208950F931F93DB
:1044E000CF93DF93EC018A019093A7028093A602F9
:1044F00040E00E94B321B801CE01DF91CF911F911E
:104500000F910C948A21FF920F931F93CF93DF9307
:1045100080E00E94E30801E008278091A802882338
:1045200081F00E94050990917D02FF24F394981375
:1045300001C0F12C11E0811110E0913021F4112320
:1045400011F010E0F12C82E10E94E3088823A9F029
:1045500082E10E944B08EC0180E00E944B08C817E2
:10456000D90728F49C012C1B3D0BE90102C0C81B94
:10457000D90BC53FD14008F001E0F11002C087E03F
:1045800001C083E080938E02112329F080918E0276
:10459000825080938E02002329F080918E028150F8
:1045A00080938E02F11004C0111102C0002311F09B
:1045B00081E001C088E00E9412320E943311811113
:1045C00002C01092A902F11008C0111106C0011119
:1045D00004C00E943311883041F08091A9028230DA
:1045E00011F481E008C082E006C08091A9028F5FCB
:1045F0008093A902F2CFDF91CF911F910F91FF908D
:1046000008950E94A62387E080938E0282E0809323
:104610008F020E940B3283E08093A902089581E00B
:104620000E94B4238FEF80938E0288E00C941232A4
:104630008093A802089581E09091AC02911180E0EE
:10464000089581E02091AA023091AB02232B09F456
:1046500080E008958091AA029091AB0208959C0198
:10466000293E8DEF380710F028EE3DEF3093AB0276
:104670002093AA02C9010E943B060C94940ABC0133
:104680008FE00E948E0C0C942F238091AC02882323
:1046900049F080E090E00E942F2381E00E945606BE
:1046A0001092AC020895CF93C82F8091AC02811173
:1046B0000BC0CC2349F080E090E00E942F2380E0E3
:1046C0000E945606C093AC02CF91089580E090E01E
:1046D0000E942F2381E00C94532381E09091B1023A
:1046E000911180E0089581E02091AF023091B002F5
:1046F000232B09F480E008958091AF029091B002DD
:104700000895482F8091AD029091AE022091AF02A2
:104710003091B0028217930711F4442341F0909333
:10472000B0028093AF020E9402070C94940A08958D
:104730009C01213080E4380710F020E030E4309311
:10474000AE022093AD0281E00C9481238091B102EE
:10475000882349F080E090E00E94982381E00E9445
:1047600049061092B1020895CF93C82F8091B102EB
:1047700081110BC0CC2349F080E090E00E94982387
:1047800080E00E944906C093B102CF91089580E075
:1047900090E00E94982381E00C94B42308958091C6
:1047A0007602873051F0982F9450943048F0815021
:1047B000823048F427EC32E008C025EB32E005C037
:1047C0002EEB32E002C020ED32E0C90108958CE109
:1047D00094E09093690280936802909176029450DD
:1047E00081E0943008F080E00E94182361E082E2CA
:1047F00094E00E94B00F91E0813009F090E0892FA1
:1048000008950F931F93CF93DF930E946B22009123
:104810007B0210917C02C0917902D0917A0263E010
:1048200086E792E00E943E19A801BE010E946E2216
:1048300086E194E0909369028093680260E087E2E9
:1048400094E0DF91CF911F910F910C94B00FEF92F4
:10485000FF920F931F93CF93DF938C01C9E7D2E0B0
:10486000E880F98061E086E792E00E943E1940E02E
:10487000B7010E94B32188819981B8010E948039D3
:10488000CB010E94C92180E194E09093690280935A
:10489000680260E083E394E0DF91CF911F910F9174
:1048A000FF90EF900C94B00FCF93DF93C0917902FB
:1048B000D0917A0261E086E792E00E943E1941E0E1
:1048C000BE010E94B32180E194E09093690280933D
:1048D000680260E083E394E0DF91CF910C94B00F25
:1048E00081E02091490330914A03232B09F480E0B1
:1048F00061E00E94162182EF93E090936902809319
:10490000680260E08FE394E00C94B00F62E086E709
:1049100092E00E943E1960917B0270917C02E091CE
:104920007D02F0917E024091590350915A03E49F19
:104930009001E59F300DF49F300D1124820F931FDD
:104940000E948A218AE094E0909369028093680231
:1049500060E08AE494E00C94B00FCF93DF93C091B1
:104960007B02D0917C0262E086E792E00E943E19D1
:10497000BE010E948A218AE094E0909369028093AC
:10498000680260E086E594E0DF91CF910C94B00F6F
:104990008CE291E0909369028093680260E08FE579
:1049A00094E00C94B00FCF93C82F8093B40224E608
:1049B00034E03093B3022093B2028D3030F4E82F0C
:1049C000F0E0E455FF4F808101C080E080936100FA
:1049D0000E946D330E94B70A0E94E723882309F4DE
:1049E0003FC084E00E941232C53049F168F4C23001
:1049F000D9F028F4CC23A9F0C13081F52CC0C33004
:104A0000B1F0C43059F516C0C83011F128F4C630E1
:104A1000C1F0C73019F519C0CB3061F0CC30F1F4DA
:104A200006C08AE090E008C00E94C82419C00E9415
:104A3000862416C085E090E00E94272411C080E003
:104A400001C081E00E9401240BC00E94702408C0B4
:104A50000E94AD2405C00E94542402C00E94AF1FD2
:104A60000E94C60ACF910C947D330F931F93CF936E
:104A7000DF93EC010E9412190E94CF238C0160E0A9
:104A8000C8010E94751887FD29C090917602E82F11
:104A9000FF27E7FDF095973019F4EB59FB4F0FC056
:104AA000892F8450843018F4E559FB4F08C0915089
:104AB000923018F4ED58FB4F02C0E858FB4F849138
:104AC0008D3049F4BE0186E792E00E94FE19CE01C6
:104AD0000E942019D1CF0E94D324D1CFDF91CF9152
:104AE0001F910F9108956BE774E08EEB92E00E94A6
:104AF00086176DE874E087EC92E00E94861769E9FA
:104B000074E085EB92E00E94861767EA74E080ED1E
:104B100092E00C948617FC014281538141155105A6
:104B200089F0A081B181B7FF03C0B195A195B1090A
:104B300028EE33E00E9452399A0140E050E00E9492
:104B4000943902C020E030E0C90108950F931F930B
:104B5000CF93DF9300D000D0CDB7DEB78C01862F86
:104B6000F801628173810E94E10A9C838B83F801C2
:104B7000808191819A838983CE0101960E948B2541
:104B80000F900F900F900F90DF91CF911F910F9189
:104B900008950F93FC01CA01002341F064177507C3
:104BA00008F4CB014617570748F409C046175707C2
:104BB00008F4CB016417750708F401C0BA019783A4
:104BC00086839183808313821282158214823387B5
:104BD0002287681B790B718760870F910895FC010C
:104BE0009B0140E050E086819781281B390B4109E9
:104BF0005109A285B3850E94593920853185442702
:104C000037FD4095542F0E94B6392115310581E0BA
:104C1000480751051CF457FD04C005C02FEF3FEFB6
:104C200002C020E030E0C9010895DF92EF92FF92C8
:104C30000F931F93CF93DF93EC012A813B812417BD
:104C4000350720F4FA01E21BF30B03C0F901E41B62
:104C5000F50B8C819D81969587958E179F0788F51A
:104C6000888199818617970720F4FB01E81BF90BCF
:104C700003C0FC01E61BF70BEF2BF9F422C08A01FD
:104C8000021B130B7B01E81AF90A06C07C01E61A25
:104C9000F70A8901041B150BC7010E947D29D82E34
:104CA000888599850E947D29D8120BC01D830C83AD
:104CB000F986E8861B870A8704C024173507F8F2AF
:104CC000E5CFDF91CF911F910F91FF90EF90DF9093
:104CD0000895CF92DF92EF92FF920F931F93CF939D
:104CE000DF93EC018B019A01A885B9850E945239A6
:104CF0002A853B8540E050E00E94B6396801E12CEE
:104D0000F12CC216D306E406F5061CF41F821E829F
:104D100004C0021B130B1F830E83DF91CF911F91E1
:104D20000F91FF90EF90DF90CF900895EF92FF9258
:104D30000F931F93CF93DF93EC018B017A010E94B5
:104D40001526A701B801CE01DF91CF911F910F91D8
:104D5000FF90EF900C9469269093400380933F035B
:104D600008958091DB02813029F420913F03309136
:104D7000400302C020E030E0C901089560913B0388
:104D800070913C038091DD020C94E10A2091E002D5
:104D9000213041F041E020913F03309140038217E0
:104DA000930708F040E0842F08952CE0829FC00113
:104DB00011246091DD0287519D4F0C94A6256091CE
:104DC000DD0281E393E00C94A625CF93DF9300D01E
:104DD00000D0CDB7DEB780E00E944B089A8389836C
:104DE00082E10E944B0829813A81281B390B3A83C2
:104DF000298386E10E944B089C838B83CE01019618
:104E00000E948B250F900F900F900F90DF91CF9104
:104E1000089590933A038093390370933C03609311
:104E20003B03CB016AE070E00E948039709340033D
:104E300060933F034093DC020895EF92FF920F933B
:104E40001F93CF93DF9391E09093DB02FF24F394C1
:104E50008F3009F0F12C8093DD0268EC70E00E9445
:104E60008E0C90933E0380933D030E944009209155
:104E70003F03309140034091390350913A030F2D85
:104E8000BC0189E293E00E94C9250E94070D80932E
:104E9000DE028091390390913A030E94500FEC0199
:104EA00010E08CE0E82E12C0812F0E94400DBC0162
:104EB00020913F0330914003E19EC00111240F2D4A
:104EC000AE018F519D4F0E94C9251F5F8091DE0268
:104ED000181750F31092E0021092DF02DF91CF9189
:104EE0001F910F91FF90EF9008950F931F93CF9311
:104EF000DF93082FEB018091DC028823C9F04091F9
:104F00003D0350913E0320913F033091400324170D
:104F1000350708F49A012C173D0710F4109264022B
:104F20008091E002813021F00E94E50E8093DB0247
:104F30008091DB02813019F58091E002823041F4EA
:104F400011E020913F0330914003C217D30708F0CE
:104F500010E00E94B1268C179D0778F0111103C054
:104F6000011101C00AC09091DF02892F8F5F8093E9
:104F7000DF0281E09A3020F402C01092DF0280E06C
:104F8000DF91CF911F910F9108950F931F93CF93AE
:104F9000DF93EC010E944009AE01BC0189E293E07D
:104FA0000E94962610E00CE00DC0812F0E94400D5B
:104FB000BC01019FC0011124AE018F519D4F0E9481
:104FC00096261F5F8091DE02181778F3DF91CF914C
:104FD0001F910F910895CF92DF92EF92FF920F935E
:104FE0001F93CF93DF936091390370913A0389E265
:104FF00093E00E94EF25EC018091390390913A03F0
:105000000E94500F7C01D12C9CE0C92E12C0CD9C77
:10501000800111240F511D4FB701C8010E94EF25D7
:10502000C817D90728F0B701C8010E94EF25EC0185
:10503000D3948091DE02D81650F3CE01DF91CF9148
:105040001F910F91FF90EF90DF90CF9008950F93F5
:105050001F93CF93DF938B01809337039093380393
:1050600020913B0330913C03EC012817390708F4E9
:10507000E9010E94B1269C018C179D0708F49E014E
:105080000217130719F18091E0028230A9F420176A
:10509000310790F080913F03909140038017910772
:1050A000A0F04091350350913603809141029091D8
:1050B00042024817590749F08091410290914202FB
:1050C000909336038093350301C09801C901DF91A5
:1050D000CF911F910F9108950F931F93CF93DF935B
:1050E000EC010E94400990932A0380932903D093F6
:1050F0002C03C0932B0310E00CE00DC0812F0E9405
:10510000400D019FF0011124EF51FD4F91838083E9
:10511000D383C2831F5F8091DE02181778F3DF917B
:10512000CF911F910F9108951F93CF93DF93182F65
:10513000EB01CB010E94C527CE010E946C280E9482
:10514000EB279093DA028093D902BE010E942728B0
:105150009C018091E002811110C0112389F080919F
:10516000DC02882321F00E94930D1092640281E0FA
:105170008093E00220E030E003C082E08093E00210
:10518000C901DF91CF911F9108950F931F93009153
:105190004103109142032091430330914403B8012D
:1051A000C9011F910F91089512BE8DE78CBF88E051
:1051B00083BF83B7836083BF89B7826089BF089547
:1051C0008091410390914203A0914303B091440325
:1051D0000196A11DB11D8093410390934203A093BA
:1051E0004303B093440308950E94E0280E94EB32E9
:1051F0000E944E2A0E94AC0480916200815019F0F6
:1052000080936200089581EE809362000E94CE2315
:105210000E9413090C945D1E1F920F920FB60F92FD
:1052200011242F933F934F935F936F937F938F93AB
:105230009F93AF93BF93EF93FF930E94F428FF9146
:10524000EF91BF91AF919F918F917F916F915F91FE
:105250004F913F912F910F900FBE0F901F90189577
:105260000F931F938FB7F89400914103109142035D
:1052700020914303309144038FBF369527951795AE
:105280000795B801C9011F910F910895CF92DF9240
:10529000EF92FF92CF93DF93EC010E9430296B01D4
:1052A0007C01CC0EDD1EE11CF11C0E9430296C1526
:1052B0007D058E059F05C8F3DF91CF91FF90EF909C
:1052C000DF90CF9008959C0180E001C08F5FF901CD
:1052D000459154912E5F3F4F452BC1F7089521E032
:1052E00030E09AE006C0A901949F9001959F300D8F
:1052F00011248150C0F7C901089597FD02C081E0D3
:1053000008958FEF0895CF92DF92EF92FF92CF939F
:105310009B01AC01611571058105910521F421E026
:1053200030E040E050E0C0E08AE0C82ED12CE12C13
:10533000F12CCF5FCA01B901A70196010E949439EF
:105340002115310541055105A1F78C2FCF91FF9013
:10535000EF90DF90CF900895BC0180E090E00C9436
:105360008329FC0180819181860F971F97FF03C0DD
:10537000118210820895242F30E0281739071CF479
:10538000408311820895918380830895FC01808178
:105390009181860F971F181619061CF081E090E086
:1053A00008C0242F30E0281739071CF440831182ED
:1053B0000895918380830895DF92EF92FF920F9377
:1053C0001F93CF93DF938C017A01DD24D3941616BB
:1053D00017060CF0D12CF801C081D181BE0180E00C
:1053E00090E00E948329823028F082500E946F2929
:1053F0009C0102C021E030E0CE01B9010E94803959
:10540000009739F0DD2019F0281B390B04C09C01EE
:105410000FC0DD2069F0C701821B930BC817D907A5
:1054200018F47901EC0EFD1EF801F182E0820BC048
:105430002C173D0718F4C21BD30B02C0C0E0D0E00C
:10544000F801D183C083DF91CF911F910F91FF901D
:10545000EF90DF9008950E9460118111FCCF0E94AF
:1054600060118823E1F30895FC01208127FD05C028
:10547000818186958F5F8170089580E00895FC0199
:10548000208127FD09C08181982F91509695282F62
:10549000269581E0921301C080E008950895089553
:1054A0006CE87EE680E00E948E0C90934603809329
:1054B00045030895CF93DF9380E00E945408209124
:1054C0004503309146032817390718F48BE195E01E
:1054D00033C086E00E944B08EC0186E00E94E3089E
:1054E000882381F18091570390915803C817D907F9
:1054F00008F128C08C179D0718F48CE295E014C0C1
:105500008091490390914A03892B11F482E027C0CE
:1055100087E00E944B0820914B0330914C032817E1
:105520003907A0F785E395E09093B3028093B20228
:1055300081E015C084E295E09093B3028093B202BB
:1055400080E00DC088E10E944B08EC0186E792E004
:105550000E945019883E2DEF920761F6D1CFDF915E
:10556000CF9108950F931F93CF93DF938C01443015
:1055700019F0CFEFDFEF02C0C1E0D0E00E9435119B
:10558000D8011B96EC91F0E0EE0FFF1FE259FE4FA1
:105590009C01C29FC001C39F900DD29F900D11240A
:1055A00020813181820F931F91838083DF91CF917E
:1055B0001F910F910895EF92FF920F931F93CF9336
:1055C000DF931F92CDB7DEB78C01443021F0EE247B
:1055D000EA94FE2C03C0EE24E394F12C69830E942C
:1055E0003511D8011B96ED91FC911C976981E60F4E
:1055F000F11DE491F0E0EE0FFF1FE259FE4F9C0118
:10560000E29EC001E39E900DF29E900D1124208138
:105610003181280F391F318320830F90DF91CF9183
:105620001F910F91FF90EF9008951F93CF93DF93F9
:10563000EC01162F0E947717CE0109960E94342A9A
:10564000882311F0298501C02FEF332727FD3095DE
:10565000812F90E02817390769F0111105C067E024
:105660008B850E94EE0C06C08B850E94420867E085
:105670000E941615DF91CF911F9108951F93CF932C
:10568000DF93EC01162F0E947717CE0109960E9436
:10569000342A882311F0898501C08FEF992787FD6F
:1056A0009095612F70E08617970741F0EB85FC8598
:1056B000E60FF71F84916D850E94EE0CDF91CF916C
:1056C0001F910895CF93DF93EC010E9486178FEF0F
:1056D000898788EA90E099838883DF91CF91089544
:1056E000CF93DF9300D000D0CDB7DEB780E00E942B
:1056F00042089A83898382E10E944B089C838B83B2
:10570000AE014F5F5F4F61E080E00E948C080F9018
:105710000F900F900F90DF91CF9108950F931F93EB
:10572000CF93DF93CDB7DEB728970FB6F894DEBFDF
:105730000FBECDBF8C0189E00E9442089E838D83FD
:1057400088E00E944B08800F911F98878F838AE022
:105750000E9442089A8389830F8118858FE10E94F5
:105760004B08800F911F9C838B83AE014B5F5F4F73
:1057700061E089E00E948C08AE014F5F5F4F61E0FD
:105780008AE00E948C0828960FB6F894DEBF0FBE00
:10579000CDBFDF91CF911F910F9108950F931F936C
:1057A000CF93DF9300D000D0CDB7DEB78C018AE075
:1057B0000E9442089A83898389E00E944B08800FE7
:1057C000911F9C838B83AE014F5F5F4F61E08AE046
:1057D0000E948C080F900F900F900F90DF91CF9147
:1057E0001F910F91089560E070E08EE395E00E94B4
:1057F000421F80E00E94E308811106C00E946011F0
:105800008130B9F780E0089581E00895CF93DF9368
:1058100000D000D0CDB7DEB7962F5A8349833C83A2
:105820002B838E3121F4C9010E948E2B0DC08F3144
:1058300021F4C9010E94CE2B07C0AE014F5F5F4F1C
:1058400061E0892F0E948C080F900F900F900F90AD
:10585000DF91CF910895FF920F931F93CF93DF9322
:10586000F62E142F022F83E00E941232812F0E9405
:105870004B08EC0181E0809340020E940E08802FCB
:105880000E944208AC019E01602F812F0E94062CCD
:105890000E940E08FF2039F0DF91CF911F910F91E8
:1058A000FF900C94702BDF91CF911F910F91FF907F
:1058B0000895CF92DF92EF92FF920F931F93CF93B1
:1058C000DF93CDB7DEB72E970FB6F894DEBF0FBECD
:1058D000CDBF0E94A6236FE475E08E010F5F1F4FBE
:1058E000C8010E94622B8DEB90E09A83898387E543
:1058F00095E09D878C8786E08E87E02ED12E61E033
:105900008E2D9D2D0E947518F82E87FD25C0082F1D
:10591000112707FD1095F801E95AFA4FC4908C2D14
:105920000E94E308882359F30E940E081092400257
:105930006F2D8E2D9D2D0E949E17882349F0F80112
:10594000E65AFA4F24914C2D60E08F2D0E942B2CAB
:1059500081E080934002D3CF81E00E94B4232E9651
:105960000FB6F894DEBF0FBECDBFDF91CF911F9170
:105970000F91FF90EF90DF90CF900895CF92DF923C
:10598000EF92FF920F931F93CF93DF93CDB7DEB7C4
:105990002E970FB6F894DEBF0FBECDBF0E94A62390
:1059A0000E94F32B882309F444C06DE575E08E0155
:1059B0000F5F1F4FC8010E94622B8DEB90E09A830E
:1059C000898381E795E09D878C8789E08E87E02E2B
:1059D000D12E61E08E2D9D2D0E947518F82E87FD29
:1059E00028C0082F112707FD1095F801EF58FA4F2E
:1059F000C49086E08F156CF38C2D0E94E3088823F9
:105A000041F30E940E08109240026F2D8E2D9D2DA5
:105A10000E949E17882349F0F801E658FA4F249116
:105A20004C2D61E08F2D0E942B2C81E08093400251
:105A3000D0CF81E00E94B4232E960FB6F894DEBF3B
:105A40000FBECDBFDF91CF911F910F91FF90EF90CF
:105A5000DF90CF9008950E94CE1181E895E00E94DA
:105A6000111365E080914703909148030E94161539
:105A70000E9495130E94D21189E895E00E941113AB
:105A800067E086E10E94EE0C0C949513EF92FF9272
:105A90000F931F93CF93DF93082F10924803109218
:105AA0004703811105C00E944523CAE7DFE304C014
:105AB0000E94A623CAEADAE00E94F32B811105C0F6
:105AC000C0E04BC0FF24F39403C0F12C5AE0E52E54
:105AD0000E942B2D0E946011182F0E9435119C01ED
:105AE000E29EC001E39E900D1124143079F44091A0
:105AF0004703509148034C175D0750F79C01240F52
:105B0000351F30934803209347030FC01230C1F470
:105B1000409147035091480348175907C8F2481B62
:105B2000590B50934803409347038091470390914A
:105B30004803011103C00E942F2302C00E94982332
:105B4000183019F4FF2021F207C0112309F4BACF4D
:105B5000113009F4B5CFBCCFC1E081E0011103C021
:105B60000E94532302C00E94B4238C2FDF91CF9157
:105B70001F910F91FF90EF900895DF92EF92FF92A7
:105B80000F931F93CF93DF9300D000D0CDB7DEB734
:105B9000162F7A01D22E0E94462D8823E9F083E049
:105BA0000E941232FC82EB828D2D0E9442089A8361
:105BB0008983AE014F5F5F4F612F8D2D0E948C084E
:105BC000802F0E9442089A838983AE014F5F5F4F06
:105BD000612F802F0E948C080F900F900F900F90D4
:105BE000DF91CF911F910F91FF90EF90DF9008957B
:105BF000FF920F931F93CF93DF93CDB7DEB7299713
:105C00000FB6F894DEBF0FBECDBF61E975E08E011F
:105C10000F5F1F4FC8010E948617F02E60E08F2D86
:105C2000912F0E947518682F87FD0DC0811103C048
:105C300042E350E002C048EE53E00FE022E080E093
:105C40000E94BD2DEBCF29960FB6F894DEBF0FBE94
:105C5000CDBFDF91CF911F910F91FF900895FF92DB
:105C60000F931F93CF93DF93CDB7DEB729970FB66E
:105C7000F894DEBF0FBECDBF67E975E08E010F5F00
:105C80001F4FC8010E948617F02E60E08F2D912FC4
:105C90000E947518682F87FD0DC0811103C042E373
:105CA00050E002C04CE251E000E123E081E00E94BC
:105CB000BD2DEBCF29960FB6F894DEBF0FBECDBF3A
:105CC000DF91CF911F910F91FF9008951F93CF9374
:105CD000DF9300D000D01F92CDB7DEB7182F6D83B1
:105CE0000E9442089A838983812F0E944B089C83DB
:105CF0008B83AE014F5F5F4F6D81812F0E948C08B7
:105D00000F900F900F900F900F90DF91CF911F91F8
:105D10000895EF92FF920F931F93CF93DF93CDB728
:105D2000DEB72C970FB6F894DEBF0FBECDBFF82EAE
:105D3000E62E6DE975E08E010F5F1F4FC8010E94CE
:105D4000622B25EC30E03A832983FC8661E0C801B0
:105D50000E94751887FD12C08111F8CF1092400281
:105D600060E0C8010E949E17882321F06E2D8F2DC0
:105D70000E94662E81E080934002E8CF2C960FB6F9
:105D8000F894DEBF0FBECDBFDF91CF911F910F9171
:105D9000FF90EF900895FF920F931F93CF93DF939F
:105DA000CDB7DEB729970FB6F894DEBF0FBECDBFD3
:105DB000F82E63EA75E08E010F5F1F4FC8010E9445
:105DC000861760E0C8010E947518682F87FD04C01F
:105DD0008F2D0E94892EF5CF29960FB6F894DEBF3D
:105DE0000FBECDBFDF91CF911F910F91FF9008950E
:105DF000FF920F931F93CF93DF93CDB7DEB7299711
:105E00000FB6F894DEBF0FBECDBF82E08093610075
:105E100069EA75E08E010F5F1F4FC8010E94861767
:105E2000F12E60E0802F9F2D0E947518182F87FD9E
:105E300029C00E946D330E94B70A123091F02CF4F1
:105E4000112349F01130C9F409C0143089F064F00D
:105E5000153099F410C00E94BE2C0FC00E94F82D7E
:105E60000CC00E942F2E09C087E00E94CB2E05C0D7
:105E70000E94483502C00E94592C0E94C60A0E9406
:105E80007D33CFCF83E08093610029960FB6F894DD
:105E9000DEBF0FBECDBFDF91CF911F910F91FF905D
:105EA000089581E00C9486370F931F93CF93DF936F
:105EB000CDB7DEB729970FB6F894DEBF0FBECDBFC2
:105EC0006EE776E08E010F5F1F4FC8010E948617B4
:105ED00060E0C8010E947518813049F0823051F0AD
:105EE00081110BC089E493E00E94CD2FF1CF0E9475
:105EF000F82EEECF0E94512FEBCF87FFE9CF2996E6
:105F00000FB6F894DEBF0FBECDBFDF91CF911F91CA
:105F10000F9108950F931F93DC015696ED91FC911C
:105F20005797EE0FFF1FEE0FFF1FE955F94F059131
:105F3000159125913491B801C9011F910F910895D0
:105F400048E150E06EE673E089E493E00E94083A8D
:105F50000C944F2A48E150E06EE673E089E493E048
:105F60000E94263A0C944F2A48E150E06BEB76E011
:105F70000C94D83989E493E00E94B42F0C94AA2F92
:105F8000FC01228533852630310520F025E030E004
:105F90003387228708950C944F2A0F931F93CF9332
:105FA000DF93CDB7DEB7A3970FB6F894DEBF0FBE71
:105FB000CDBF8C01BC01CE0101960E94FA2FCE010B
:105FC00001960E94173088E1FE013C96D8010190AD
:105FD0000D928A95E1F70E94AA2F0E944F2AA3965C
:105FE0000FB6F894DEBF0FBECDBFDF91CF911F91EA
:105FF0000F9108950F931F93CF93DF93EC018B01C3
:1060000063ED76E00E9486178FEF89878DEC90E034
:106010009983888388E1F801DE011B9601900D9237
:106020008A95E1F7DF91CF911F910F910895DF924B
:10603000EF92FF920F931F93CF93DF93CDB7DEB70D
:1060400068970FB6F894DEBF0FBECDBF7C0188E124
:10605000D82E8701055F1F4F60E0C7010E947518A9
:1060600087FD2AC08D3039F4C8010E94B42F83E027
:106070000E941232F1CFF801DE0111969D2D0190A0
:106080000D929A95E1F7682FC7010E949E17811122
:1060900009C0FE013196D8018D2D01900D928A958F
:1060A000E1F706C083E00E941232C8010E94C02FAF
:1060B000C8010E94CB2FD0CF68960FB6F894DEBFF0
:1060C0000FBECDBFDF91CF911F910F91FF90EF9049
:1060D000DF90089564E670E00E948039CB0163E0B0
:1060E0000E94161583E40C946B1368EE73E00E9413
:1060F0008039CB0163E00E94161586E50C946B1382
:10610000CF93DF9364E670E00E9480399B01EC013D
:1061100063E0C9010E9416158EE20E946B13CE0146
:106120006AE070E00E948039862F0E9498138FEEFB
:1061300096E0DF91CF910C941113DC015F96ED9105
:10614000FC919097EE0FFF1FED50F94F2591349180
:10615000C9010C9411130B960E948A2F24E630E09B
:1061600040E050E00E94943965E0C9010E94161594
:1061700080E30E946B1380E30C946B131F93CF9307
:10618000DF93EC01162F0E947717CE0109960E942B
:10619000342A882311F0298501C02FEF332727FDEA
:1061A0003095812F90E02817390709F459C0153030
:1061B000A9F178F4123029F130F41123C9F011302B
:1061C00009F04EC019C0133009F1143009F048C06D
:1061D00021C01830A1F130F4163031F1173009F038
:1061E0003FC028C01A30A9F170F11B30C9F535C085
:1061F0008B850E94621334C08D859E850E946A3013
:106200002FC08F8598890E9480302AC065E08989D7
:106210009A891CC065E08B899C8918C063E08D89D0
:106220009E890E9416151CC065E08F89988D0E947A
:10623000441516C0898D9A8D0E94753011C066E094
:106240008B8D9C8D03C065E08D8D9E8D0E944D15BC
:1062500007C0CE010E949D3003C0CE010E94AB302A
:10626000DF91CF911F910895FC0124E6269FC00184
:10627000279F900D112420813181820F931F843636
:10628000910508F002C084E690E0918380838081CC
:1062900091818D3A964220F08CEA96E29183808338
:1062A0000895FC012AE0269FC001279F900D11242C
:1062B00020813181820F931F8A30910508F002C03E
:1062C0008AE090E09183808380819181893E934030
:1062D00020F088EE93E0918380830895FC0128EEFE
:1062E00033E0629FC001639F900D729F900D112457
:1062F00020813181820F931F88352BE1920708F0AE
:1063000002C088E59BE19183808380819181813304
:10631000954720F080E395E7918380830895FC0101
:1063200080819181680F791F6330710518F0718346
:10633000608304C083E090E09183808380819181B9
:10634000893C910520F088EC90E09183808308954A
:10635000262F443019F06FEF7FEF02C061E070E04C
:10636000253059F168F42230F9F028F42223B1F0F5
:106370002130E1F516C02330D1F02430B9F51AC030
:10638000283029F128F42630D9F0273079F51CC0BF
:106390002A3029F108F12B3049F524C041E00B9651
:1063A00023C00D960C9434310F960C94513144E176
:1063B00041961AC044E1439617C045E0459602C095
:1063C0004AEF47960C94C62949960C946E3148EED4
:1063D00053E04B960C94DC294D960C948F3144E09D
:1063E0004F9602C044E081960C94B1290895CF9352
:1063F0000E94CB0AC82F882349F080916103811144
:1064000002C00E94BD1F87E00E941232C093610348
:106410008C2FCF9108950E94C528709366036093D6
:106420006503089590916203981721F080936203A9
:106430000C940B32089588E00C9412329091620310
:10644000983011F40C94123208959B01220F331FDF
:10645000281739075CF0681779071CF4281B390BDB
:1064600007C01816190614F49C0102C020E030E0A1
:10647000C9010895969587958531910520F46AE0C4
:1064800070E00C9425320E941B3280E090E0089569
:106490000F931F93CF93DF93EC01D695C795D695B5
:1064A000C795C93CD1052CF00E941B3220E030E09A
:1064B0000FC06AE070E0CE010E9425328C016AE0D4
:1064C00070E0CE0188970E9425329C01200F311F79
:1064D000C901DF91CF911F910F91089560ED77E091
:1064E0000E9480396AE070E00C9425326AE070E026
:1064F0000E948039CB016D38710520F464E170E0B1
:106500000C9425320E941B3280E090E008956AE0EE
:1065100070E00E9480399B01CB0168E270E00E942C
:106520008039283B314020F464E170E00C9425323E
:106530000E941B3280E090E008956AE070E00E94C3
:1065400080399B01CB0168E270E00E9480392135DF
:10655000310520F464E170E00C9425320E941B3276
:1065600080E090E008956AE070E00E9480399B012D
:10657000CB0168E270E00E948039283B314020F472
:1065800064E170E00C9425320E941B3280E090E0C0
:106590000895209162032330A9F020F4213061F0A6
:1065A00068F408C0253061F068F0263079F02730B3
:1065B00079F40AC00C943A320C946E320C94763210
:1065C0000C9487320C9448320C949D320C94B33264
:1065D00080E090E008950E94C528209165033091E5
:1065E0006603CB01821B930B0E94C9322091630387
:1065F000309164038217930731F090936403809382
:1066000063030C94D0040895CF93DF931F92CDB70A
:10661000DEB7E0919F04F091A004309729F4E3EAFB
:10662000F4E002C0219303C0CE0101962EEB8E1739
:106630009F07C0F70F90DF91CF910895CF93DF931D
:1066400000D0CDB7DEB780919F049091A004009751
:1066500011F483EA94E09E012F5F3F4F281B390B12
:10666000C9010F900F90DF91CF910895CF93DF93E1
:106670001F92CDB7DEB720919F043091A004211561
:10668000310511F423EA34E0F901CE010196AF019E
:10669000421B530B8E179F0728F060816E3B11F44D
:1066A0003196F5CFCA010F90DF91CF91089589E41B
:1066B00093E00E948A2FAB01BC0180E793E00C9429
:1066C000593680E793E00E94A03580E793E00E946E
:1066D000CE3660E08AE00C94AE3880916300813061
:1066E00059F480915D0390915E03892B29F00E94FB
:1066F000573382E080936300089580916300813076
:1067000029F00E94613381E0809363000895CF9364
:10671000C82F682F80E793E00E941F38909167038D
:106720009C2790936703CF9108958BE30C94873354
:10673000CF93DF93EC0102C00E94873389918111CE
:10674000FBCFDF91CF9108950F931F93CF93DF93EA
:10675000CDB7DEB72B970FB6F894DEBF0FBECDBF17
:106760008E010F5F1F4F1A87098727E02B87AC0127
:10677000BE01655F7F4FCE0109960E942E12C801AF
:106780000E9498332B960FB6F894DEBF0FBECDBF94
:10679000DF91CF911F910F910895CF93DF93EC017B
:1067A0001092670384E20E948733CE010E94A433D3
:1067B0000E9495338091610090E00E94A4330E9472
:1067C0009533609168037091690380916A03909199
:1067D0006B0328EE33E040E050E00E949439C90199
:1067E0000E94A4338EE20E94873360916803709107
:1067F000690380916A0390916B0324E630E040E0E6
:1068000050E00E949439CA01B9012AE030E040E02A
:1068100050E00E949439CB010E94A433DF91CF91C4
:106820000C9495338DE00E9487338AE00C94873373
:106830008091670390E00E94A4330C941234CF93AC
:10684000DF9381E090E00E94CD33C0E0D0E0FE0114
:10685000ED55F84F84910E944B080E94A4330E948A
:1068600095332196CE30D10591F7C0E08C2F0E9450
:10687000D5260E94A4330E949533CF5FC630B1F76E
:106880000E94DF260E94A4330E9495330E94E526D1
:106890000E94A4330E949533DF91CF910C94183459
:1068A000CF93DF93D82F82E090E00E94CD33C0E0F9
:1068B0008C2FDD2319F00E94420802C00E944B0871
:1068C0000E94A4330E949533CF5FC43289F7809130
:1068D000650290E00E94A4330E9495330E94D20585
:1068E0008091D9029091DA020E94A4330E949533DC
:1068F000DF91CF910C94183483E090E00E94CD3367
:106900000E9436330E94A4330E9495330E941E33A6
:106910000E94A4330E9495330C941834CF93DF93D4
:10692000C0915D03D0915E030E941F34C230D10537
:106930006CF081E0C430D1050CF480E00E9450344A
:10694000229721F0DF91CF910C947C34DF91CF918D
:1069500008950F931F9380916300813051F10E943D
:10696000302920916300223051F460936C037093BE
:106970006D0380936E0390936F03109263000091F8
:106980006C0310916D0320916E0330916F03DC0155
:10699000CB01801B910BA20BB30B809368039093E8
:1069A0006903A0936A03B0936B031F910F910C943A
:1069B0008E341F910F9108950F931F93CF93DF9300
:1069C0001F92CDB7DEB78A0169830E948733698140
:1069D000862F90E00E94A4338DE30E948733C80184
:1069E0000E94A4330F90DF91CF911F910F910C94CF
:1069F00012341F93CF93DF9300D000D0CDB7DEB712
:106A000081ED90E00E9498330E94123447E050E0FC
:106A100060E085E40E94DC3441E050E061E085E420
:106A20000E94DC3442E050E062E085E40E94DC3405
:106A300010E040E0612FCE0101960E946E0849816E
:106A40005A81612F81E60E94DC344B815C81612F89
:106A500082E70E94DC3441E0612FCE0101960E9462
:106A60006E0849815A81612F81E40E94DC344B8198
:106A70005C81612F82E50E94DC341F5F1131C9F611
:106A80000F900F900F900F90DF91CF911F9108956D
:106A90000E9457330E94F9340E9412340E94F93444
:106AA0000E9412340C946133FC0184859585FC01AD
:106AB000F39520813181FC01EE5FFE4F8081918151
:106AC000281B390B3327C9010895FC01848595855E
:106AD000FC01F39540815181FC01EE5FFE4F208166
:106AE00031814217530741F00190F081E02DE80F0A
:106AF000F91F208130E002C02FEF3FEFC901089558
:106B0000FC0184859585FC01F39540815181FC0150
:106B1000EE5FFE4F208131814217530769F0A0815B
:106B2000B181A80FB91F2C9180819181019699277D
:106B30009183808330E002C02FEF3FEFC9010895B9
:106B4000FC0181A1882329F0A489B5898C9186FF55
:106B5000FBCF11A20895CF93DF93FC0126853785E3
:106B6000D901B3958D919C91119701969927E901CF
:106B7000CE5FDE4F4881598184179507D9F30D9078
:106B8000BC91A02DA20FB31F6C93A685B785B395BA
:106B900011969C938E93A689B7892C9181E090E001
:106BA000078C02C0880F991F0A94E2F7282B2C93B8
:106BB00081E081A30488F589E02D80818064808351
:106BC00081E090E0DF91CF91089508951F920F9298
:106BD0000FB60F9211242F933F934F938F939F9350
:106BE000EF93FF935A991AC04CB1809192049091FF
:106BF000930401969927209194043091950482176B
:106C0000930769F0E0919204F0919304EE56FC4FE3
:106C10004083909393048093920401C08CB1FF91C0
:106C2000EF919F918F914F913F912F910F900FBEB8
:106C30000F901F90189580E793E00E945435892BA0
:106C400011F00C94E53508951F920F920FB60F9234
:106C500011242F933F938F939F93EF93FF93209152
:106C60009204309193048091940490919504281794
:106C7000390711F4559812C0E0919404F0919504ED
:106C8000EE56FC4F208180919404909195040196DA
:106C9000992790939504809394042CB9FF91EF91D8
:106CA0009F918F913F912F910F900FBE0F901F904A
:106CB0001895CF92DF92EF92FF92CF93DF93EC0182
:106CC0006A017B01411581EE580761057105F9F0F4
:106CD000EC89FD8981E090E008A002C0880F991F2F
:106CE0000A94E2F7808360E079E08DE390E0A70109
:106CF00096010E9494392150310941095109569554
:106D0000479537952795211580E1380798F0EC894C
:106D1000FD89108260E874E88EE190E0A701960199
:106D20000E949439215031094109510956954795DE
:106D300037952795E889F9893083EA89FB8920838B
:106D400019A2EE89FF89408181E090E09C010D8CC1
:106D500002C0220F331F0A94E2F7422B4083EE89D0
:106D6000FF8940819C010E8C02C0220F331F0A94C0
:106D7000E2F7422B4083EE89FF8920810F8C02C00D
:106D8000880F991F0A94E2F7809582238083DF9110
:106D9000CF91FF90EF90DF90CF900895CF93DF9346
:106DA000FC0186859785DC01B395EC01CE5FDE4F53
:106DB0004D915C9111972881398142175307C1F792
:106DC000A689B7894C9181E090E09C01058C02C0B6
:106DD000220F331F0A94E2F7209524232C93A689CF
:106DE000B7894C919C01068C02C0220F331F0A9474
:106DF000E2F7209524232C93A689B7892C91078C40
:106E000002C0880F991F0A94E2F7809582238C9321
:106E100084859585FC01EE5FFE4F20813181FC0168
:106E2000F39531832083DF91CF91089510927303FE
:106E30001092720388EE93E0A0E0B0E080937403B8
:106E400090937503A0937603B09377038CED90E055
:106E5000909371038093700382E993E090937D0394
:106E600080937C0390937F0380937E0380E490E083
:106E7000909381038093800329E230E03093830371
:106E8000209382032BE230E0309385032093840328
:106E90002AE230E03093870320938603909389039E
:106EA000809388038CE290E090938B0380938A0315
:106EB00084E080938C0383E080938D0387E080934C
:106EC0008E0385E080938F0381E080939003089583
:106ED0000F931F93CF93DF9300D0CDB7DEB78C0114
:106EE00069837A830E94203A69817A81861797079D
:106EF00029F0C8010E94473A81E001C080E00F906C
:106F00000F90DF91CF911F910F910895CF93DF9351
:106F1000C82F62EC77E081EB97E00E94421F67E0A8
:106F200070E080E090E00E94683781111DC0C111BF
:106F30001BC061E070E08AE890E00E946837811130
:106F40001BC0C11119C0D0E062E070E08CE693E094
:106F50000E946837811118C0D11116C0CC23F9F0F6
:106F6000DF91CF910C94B31F8CEC97E00E9411132A
:106F70000E94A308C1E0DDCF8FEC97E00E941113BF
:106F80000E94041BD1E0E0CF82ED97E00E94111334
:106F90000E94BA2F80ED97E00E944629DFCFDF9153
:106FA000CF9108950E947D380E943F10CBE1D6E337
:106FB0000E942D102097E1F30E941B36F9CFCF924B
:106FC000DF92EF92FF920F931F93CF93DF936C01A9
:106FD000EB017A01E60EF71E00E010E00BC06991AC
:106FE000D601ED91FC910190F081E02DC60109954B
:106FF000080F191FCE15DF0591F7C801DF91CF915A
:107000001F910F91FF90EF90DF90CF900895611541
:10701000710581F0DB010D900020E9F7AD014150D1
:107020005109461B570BDC01ED91FC910280F38165
:10703000E02D099480E090E008950C940738DC017D
:10704000ED91FC910190F081E02D09948093640012
:1070500008951F920F920FB60F9211242F933F9312
:107060008F939F93AF93BF938091960490919704D1
:10707000A0919804B091990430919E04232F2D5F24
:107080002D3720F40196A11DB11D05C0232F2A57CD
:107090000296A11DB11D20939E04809396049093A7
:1070A0009704A0939804B093990480919A049091C6
:1070B0009B04A0919C04B0919D040196A11DB11D5B
:1070C00080939A0490939B04A0939C04B0939D0496
:1070D000BF91AF919F918F913F912F910F900FBED4
:1070E0000F901F901895019739F0880F991F880FFE
:1070F000991F02970197F1F70895789483B78260FA
:1071000083BF83B7816083BF89B7816089BF1EBC9D
:107110008EB582608EBD8EB581608EBD8FB581606B
:107120008FBD85B5846085BD85B5806485BD329A87
:10713000319A309A379A1AB80895843039F08530E8
:1071400049F0833051F48FB58F7702C08FB58F7DB2
:107150008FBD089585B58F7D85BD0895CF93DF934D
:1071600090E0FC01EE5FF74F4491FC01E15DF74FC9
:107170008491882341F190E0880F991FFC01E05928
:10718000F74F25913491D9018A59974FFC01859188
:107190009491C82FD92F9FB7F8948C91611106C094
:1071A000409584238C938881842308C0623041F405
:1071B000242F209582238C938881842B888302C07E
:1071C000842B8C939FBFDF91CF9108950F931F93D2
:1071D000CF93DF931F92CDB7DEB7282F30E0F901B0
:1071E000EB52F84F8491F901EE5FF74F1491F901DA
:1071F000E15DF74F04910023D1F0882321F06983EA
:107200000E949D386981E02FF0E0EE0FFF1FEA59E0
:10721000F74F85919491DC019FB7F8948C9161119F
:1072200003C01095812301C0812B8C939FBF0F90C9
:10723000DF91CF911F910F910895CF93DF93282F66
:1072400030E0F901EB52F84F8491F901EE5FF74F0E
:10725000D491F901E15DF74FC491CC2389F08111FC
:107260000E949D38EC2FF0E0EE0FFF1FE45AF74F1D
:1072700085919491DC018C918D2321E030E011F413
:1072800020E030E0C901DF91CF910895A29FB001C5
:10729000B39FC001A39F01D0B29F700D811D112427
:1072A000911D08950E944639B7FF0895821B930BE4
:1072B00008950E944639A59F900DB49F900DA49FFC
:1072C000800D911D11240895DB018F939F930E94DF
:1072D0005939BF91AF91A29F800D911DA39F900D31
:1072E000B29F900D11240895991B79E004C0991F55
:1072F000961708F0961B881F7A95C9F78095089510
:10730000AA1BBB1B51E107C0AA1FBB1FA617B707CB
:1073100010F0A61BB70B881F991F5A95A9F78095E7
:107320009095BC01CD010895A1E21A2EAA1BBB1BAA
:10733000FD010DC0AA1FBB1FEE1FFF1FA217B30741
:10734000E407F50720F0A21BB30BE40BF50B661F57
:10735000771F881F991F1A9469F76095709580951B
:1073600090959B01AC01BD01CF010895052E97FBBF
:1073700016F4009407D057FD0DD00E94943907FCF5
:1073800009D07EF490958095709561957F4F8F4FD1
:107390009F4F089550954095309521953F4F4F4F01
:1073A0005F4F0895EE0FFF1F0590F491E02D0994B3
:1073B000FB01DC0102C005900D9241505040D8F70E
:1073C0000895FC0105900020E9F7809590958E0FB7
:1073D0009F1F0895FB01DC014150504048F005908B
:1073E0000D920020C9F701C01D9241505040E0F7B6
:1073F0000895FB01DC014150504048F001900D928E
:107400000020C9F701C01D9241505040E0F7089597
:10741000DC01CB01FC01E199FECF06C0FFBBEEBB56
:10742000E09A31960DB20D9241505040B8F7089550
:10743000E199FECF9FBB8EBBE09A99278DB308954B
:10744000A8E1B0E042E050E00C940A3ADC01A40F5D
:10745000B51F4150504048F0CB01840F951F2E912D
:107460000E94373A41505040D0F70895262FE199B5
:10747000FECF9FBB8EBBE09A01970DB2021631F092
:107480002DBB0FB6F894E29AE19A0FBE08950196CB
:0E749000272F0E94373A0C94363AF894FFCF1B
:10749E00FF03E10101000040001400540000000150
:1074AE0002010201010101010101000005010101BA
:1074BE000100000000001D10000000004616DF371E
:1074CE0000000000771700000000E8170000000021
:1074DE00691B441B00000000421B431B05060807E6
:1074EE00050909050700000507000000003E2BDB1B
:1074FE002A00000000152BB22A00000000BE30A8A2
:10750E0031563D302E33320000000000AB35DF37F0
:08751E00543580356535A035B8
:00000001FF
